:020000040800F2
:103000000080002075C40008858D0008C18D00086F
:1030100000000000000000000000000000000000B0
:10302000000000000000000000000000ABC4000829
:103030000000000000000000ADC400086D02002088
:103040007BC400087DC400087FC4000881C4000858
:1030500083C4000885C4000887C4000889C4000828
:103060008BC400087D0200208DC400088FC40008B6
:10307000DD02002091C4000893C4000895C4000834
:1030800097C40008218E0008318E0008418E000888
:1030900099C40008518E0008618E00089BC4000886
:1030A0009DC400089FC40008A1C400084903002073
:1030B000A3C40008A5C40008A7C40008A9C4000848
:1030C000014802490160704708ED00E00030000847
:1030D000B0B51E4D2C1F20688006400F411E0329ED
:1030E00022D81B487944097949008F442301171AD3
:1030F000296803220A40032A00D016482968490695
:10310000490F491C08F098FF29684904490E4843B3
:103110002968490F491C08F08FFF0BE07D20000251
:1031200008E00120C00305E00C3D28688004410F41
:103130000848C84008498864226892093C23134023
:10314000064AD258D0408864B0BDC0460C10024038
:1031500000127A000024F400E4050020B0C3000847
:1031600000B5CFB03C25E04801264655A7204100D8
:103170002C914E39DD4A10681E91084310607D2065
:103180001790C100DA48806C349108F055FF401E5A
:10319000010E320726920322299293070029D54F68
:1031A00031D1D5494860D54A1068D54C20401843E4
:1031B0001060002088600720086010682040D14916
:1031C0001831014311604420C7490E54386C304314
:1031D0003864386C30403D903D98F86B2699084330
:1031E000F863F86B08403D903D98C7480168B143CB
:1031F0000160016802220A430260C449EC313038A0
:1032000002680A430260249329984002C04C214678
:1032100014390A6882430123580225901018086067
:10322000B348816C379398023690206840057FD46C
:103230002F963595B868F968299A8A4338213391D1
:10324000084010230146329359408A185142514197
:10325000379A920331920828386829D0002927D15B
:10326000AC49C91F0843386037984004AA490A6A24
:103270003B6803421CD10B6A9B1A642B00D981E185
:103280003B68034214D10B6A9B1A642B00D979E185
:103290003B6803420CD10B6A9B1A642B00D971E185
:1032A0003B68034204D10B6A9B1A642BE0D969E1A5
:1032B000B968339801400A4632984240FB680320BF
:1032C000034002245C401219534253413A680029DA
:1032D00061D0002B5FD10721C9028A43C0021018B8
:1032E000386038681E99084338608B48016A3A682C
:1032F000369B1A425BD1026A521A022A00D941E176
:103300003A681A4253D1026A521A022A00D939E1A4
:103310003A681A424BD1026A521A022A00D931E1A4
:103320003A681A4243D1026A521A022ADFD929E1C5
:1033300006204843794908F07FFE0221081A032835
:1033400000D175E7821E514251412268369B1A42D4
:10335000324600D00A46002A00D069E7421E514298
:1033600051412268369B1A42324600D00A46002A52
:1033700000D05DE7414241412268369B1A42324605
:1033800000D00A46002A00D052E7001D2168369A74
:103390001142D4D14CE77F2212027B689343319AC9
:1033A00013437B6000290AD05148806C15E07F20D0
:1033B00000027968814331980143796037E0072141
:1033C000C9023A688A43C00210183860386880041D
:1033D000410F5348C84046498864434944240E5D20
:1033E000002E01D1354601E0464D1835349908F0DC
:1033F00023FE401E4249884200D9C3E03E4948604E
:103400003E4A10683E4B1840249B18431060002031
:10341000886007200860002E00D1B3E011460868DC
:10342000374A1040284308602F482F990155B86843
:10343000339908401828386E0CD1B8683399084081
:1034400010282BD1F868374901403748814200D015
:1034500098E0ACE00121084338662F48016A3A6ED3
:103460009207EAD4026A521A022A00D98AE03A6E16
:103470009207E2D4026A521A022A00D982E03A6E16
:103480009207DAD4026A521A022A7BD83A6E92075D
:10349000D3D4026A521A022AE1D973E0012001064C
:1034A0003A688A433A6040061B490A6A3B6803420D
:1034B0003CD00B6A9B1A022B64D83B68034235D080
:1034C0000B6A9B1A022B5DD83B6803422ED00B6A15
:1034D0009B1A022B56D83B68034227D00B6A9B1AD3
:1034E000022BE3D94EE0C046281100200020024004
:1034F000E40500200010024010E000E020ED00E0B4
:10350000FFFFFF00E8FFFF7F3000014014050000CF
:103510001470004007000100A411002040420F0079
:103520000024F400737F3EEE03100222FA68E84B99
:103530001340E84A9A18FA60E74A521C3B68134362
:103540003B60FA68269B1A43FA600A6A3B680342AA
:103550002DD10B6A9B1A022B14D83B68034226D14B
:103560000B6A9B1A022B0DD83B6803421FD10B6AD2
:103570009B1A022B06D83B68034218D10B6A9B1A90
:10358000022BE3D90026F149304608F0C9FEF04984
:10359000304608F0C5FEEF49304608F0C1FEEE495E
:1035A000304608F0BDFEED49304608F0B9FE3798C8
:1035B000C0032190EA4800684007800F00D18DE1E8
:1035C00007263003E74B9968014399600F210902F0
:1035D0009A688A439A601968890100D53CE1002500
:1035E000DA49284608F09CFED949284608F098FE9A
:1035F000D849284608F094FED749284608F090FE9E
:10360000D649284608F08CFE379CE004D54A11685C
:103610000143116000254195506B0421084350631C
:10362000506B1F9108404A904A98506B20212E9170
:1036300008435063506B08404A904A98506B2043AF
:103640005063506B20404A904A98506B022134914D
:1036500008435063506B08404A904A98506B0821C9
:1036600008435063506B289108404A904A98600381
:10367000BD4E1190B0613198B062BC493F20886165
:103680000520139001072291E0022B908862B84830
:103690002999816240953F953E9448033D903DAF06
:1036A0003046394606F054FF3F953E9521983D90AF
:1036B0003046394606F04CFF40953F953E941F201A
:1036C00015903D90A948103806463090394606F0CE
:1036D0003FFF3F943E95FF201D90000210903D90CB
:1036E0003046394606F034FF3F953E951E983D9092
:1036F000229E3046394606F02BFF3F943E95C0206F
:103700003D909948394606F023FF299840903F950F
:103710003E942B983D903046394606F019FF3F9471
:103720003E9521983D903046394606F011FF409570
:103730003F953E943D948E48394606F009FF299EF8
:103740003EA870C034983D908948394606F000FF85
:103750003F943E950C202D903D908548394606F0CB
:10376000F7FE3EA870C02E983D903098394606F07E
:10377000EFFE7C4FB86B2043B86330037D4B239042
:103780001862802140227C48183021C3319818608B
:1037900012925A602A9199602598D8602B981861E6
:1037A0005D61B86B20403D903D98083B184606F09F
:1037B00083FC002814D000266449304608F0B0FD90
:1037C0006349304608F0ACFD6249304608F0A8FD78
:1037D0006149304608F0A4FD6049304608F0A0FD7C
:1037E000664A106866490840319908431060654987
:1037F00025980860644935980D542C201B900C5472
:10380000CD642003279008634C63349888634D622D
:103810008D62081D057706201490C8618C760D8393
:103820006205A007594E0E60209048608D60CD6003
:103830001C920A612846289D4D613A903990389033
:1038400030903B90886D002800D1A5E0B068269F9D
:10385000384200D11EE145E11A46916802233093B7
:1038600019430524A143916049490D6A494A3D4BDA
:103870009F68339B1F40102F00D1F2E10F6A7F1B1E
:10388000974200D9ABE6374B9F68339B1F40102F00
:1038900000D1E6E10F6A7F1B974200D99FE6314BCA
:1038A0009F68339B1F40102F00D1DAE10F6A7F1B06
:1038B000974200D993E62B4B9F68339B1F40102FF4
:1038C00000D1CEE10F6A7F1B9742D0D987E6C04670
:1038D0008C80C11103100222FFFFFF00204A1068F4
:1038E000022101430520814311602948016A294AC8
:1038F0001B4B1C6807231C40022C00D160E6046AA5
:10390000641A944200D96AE6154C24681C40022CC3
:1039100000D155E6046A641A944200D95FE6104C5F
:1039200024681C40022C00D14AE6046A641A9442BE
:1039300000D954E60A4C24681C40022C00D13FE612
:10394000036A5B1A9342D3D949E6C046CCD000083B
:1039500042CC000881C900082CC9000840CC0008EE
:1039600000200240001002400008005010040050E7
:10397000000C0050781200200400024008E400E02F
:10398000FF00FFFF00E100E01412002000240140CE
:10399000A41100208813000000244E944D943DAEE5
:1039A000301D302108F0D0FB31983D90304606F0B4
:1039B0000FFF002814D00026F149304608F0B0FC73
:1039C000F049304608F0ACFCEF49304608F0A8FC5E
:1039D000EE49304608F0A4FCED49304608F0A0FC62
:1039E00001200105EB4B1A6C0A431A641A6C0A4059
:1039F0003C923C99596B01435963596B01403C918E
:103A00004C9403204B90CF204A903C984AA922988E
:103A100006F09EFDE04E239830620520DF49091D27
:103A200031607060B460F4602A9830611E987061F3
:103A30003698B0612E98F061304606F03DFB0028C4
:103A400014D00027CE49384608F06AFCCD493846E4
:103A500008F066FCCC49384608F062FCCB49384691
:103A600008F05EFCCA49384608F05AFCCC4AB262FB
:103A70001665CC4B58681D9988435860CA482799E9
:103A8000016054201454D4651668379CB068269F92
:103A9000384227D1B068C54901403943B160C448B4
:103AA000806CC44908F0C8FA4000801C3B903B98E9
:103AB000002817D03B98401E3B903B98002811D01F
:103AC0003B98401E3B903B9800280BD03B98401EF3
:103AD0003B903B98002805D03B98401E3B903B987C
:103AE0000028E7D1B0683840AD4F329B06D1B96DA0
:103AF0001943B965F96D01220A43FA65B1681F9A45
:103B00001140BA6D1A405118E24326920029B96D4E
:103B10006CD1812252009143891CB965B168C907F3
:103B2000309931D1F168182291437A68BB680B4310
:103B3000F360249B1340F96C1943359BFB5C012B0C
:103B400007D13B6C19437B6C0B43BC6C1C430121BC
:103B500021433369984C1C400C4334610123DC073A
:103B6000A24211D00324A407A2420DD09B079A427F
:103B70000AD00F239B041A40904B5B1E904C276881
:103B80001F40BA18864F22603B6B002B279A00D14A
:103B90001A463B7E9B037C7E3D46E7031F43AC7E7B
:103BA00063033B43EF681F4317432B69002B1C9AA9
:103BB00002DA844A17321A401743794D1B9AAA5CDD
:103BC00052003A432E9FEF5D012F12D1002C00D1FD
:103BD000B1E0734DAC6D2E9F3C43AC65EC6D01279D
:103BE0002743EF656C6A002C07D10CE01943B965D7
:103BF00002E16B4D6C6A002C05D02C9F72373C4063
:103C00001443AA6A2243F4686F4F27401743F760B2
:103C100034696E4F27400F43376171690724A14310
:103C20006C6B0C43746171697024A143AC6B24010B
:103C30000C437461002B2F4646D0012149058B426D
:103C4000289D379C00D08AE0396E0F230B400F2B44
:103C5000B36A79D0F0240C40F02C75D126990E3936
:103C60007AE05B4B1D683540032D34D31D68309FCF
:103C70003D43A5431D600B6A554C24683440022C1B
:103C800029D00C6AE41A944200D9A8E4504C246864
:103C90003440022C1FD00C6AE41A944200D99EE4EE
:103CA0004B4C24683440022C15D00C6AE41A944220
:103CB00000D994E4464C24683440022C0BD00C6AA2
:103CC000E41A9442D8D98AE426990E39B36A0B4390
:103CD000B362289D42E02F4DA9688143A960A8687E
:103CE0008006400F01D101F0E5F8A868339A104032
:103CF00008283848359C01D101F0E2F8A968114044
:103D0000102901D001F016F9E96803220A40032ABC
:103D100000D03148E9684906490F491C08F08CF980
:103D2000E9684904490E4843E968490F491C08F00D
:103D300083F901F0C5F8294CE41F2243184D6C6A41
:103D4000002C00D059E75EE7FB699B001C331C2464
:103D50001C40269B0E3BA3400B43B362379CF1688B
:103D60001F4B0B4093423DD10021F965B96D0122F3
:103D70000A4302218A43BA6500283DD051E0C0467B
:103D8000CCD0000842CC000881C900082CC900082A
:103D900040CC000800100240D41200200400024071
:103DA0001412002008E400E000E100E0E8FFFF6FEB
:103DB000E4050020400D030002FCFF1F0000C4FFCB
:103DC00008270140E8FFFF7F1902FEFF02FCFFDF2A
:103DD0000020024000127A000024F40007000100D5
:103DE000E7FF3F83B86D3299084302218843B865E5
:103DF000F86D01210143F9650026E149304608F0DC
:103E00008FFAE049304608F08BFADF49304608F077
:103E100087FADE49304608F083FADD49304608F07B
:103E20007FFADC483A9030983990389438A805F0F9
:103E300081FD002814D00026D149304608F070FAE0
:103E4000D049304608F06CFACF49304608F068FA9D
:103E5000CE49304608F064FACD49304608F060FAA1
:103E600030983A901F983990CB48389038A805F090
:103E700061FD002814D00026C149304608F050FAF0
:103E8000C049304608F04CFABF49304608F048FABD
:103E9000BE49304608F044FABD49304608F040FAC1
:103EA0003995BE48389038A805F044FD00282A9F6F
:103EB00014D00026B249304608F032FAB1493046F3
:103EC00008F02EFAB049304608F02AFAAF493046D9
:103ED00008F026FAAE49304608F022FA2D983990BB
:103EE000AF48389038A805F025FD0028309D14D043
:103EF0000026A349304608F013FAA249304608F0DC
:103F00000FFAA149304608F00BFAA049304608F0F4
:103F100007FA9F49304608F003FA32983990A148D1
:103F2000389038A805F006FD002814D000269449E2
:103F3000304608F0F5F99349304608F0F1F9924916
:103F4000304608F0EDF99149304608F0E9F990491A
:103F5000304608F0E5F9142039909348389038A895
:103F600005F0E8FC002814D000268549304608F00A
:103F7000D7F98449304608F0D3F98349304608F030
:103F8000CFF98249304608F0CBF98149304608F034
:103F9000C7F9864C864825626562A562E12149021F
:103FA00003C42799216065603699A1602D99E1606D
:103FB000256165618422083CA1580029249205D11D
:103FC000E55504F055FF249A784C2068242123916C
:103FD000A1500168379A9143016006F04FFF012814
:103FE00030D0A06A002802D007F038F96F4C206862
:103FF0008168319A11438160379BD90382688A4373
:10400000826001686B4A0A400260016819430160DE
:104010008C21655068490E6A0168090707D51C980C
:10402000314607F087F90028604C0BD12068006802
:1040300040075E4C68D537988005314607F07AF91D
:10404000002861D000264E49304608F069F94D49F4
:10405000304608F065F94C49304608F061F94B49A3
:10406000304608F05DF94A49304608F059F9E05DFC
:104070000128224650D100244149204608F050F939
:104080004049204608F04CF93F49204608F048F9DD
:104090003E49204608F044F93D49204608F040F9E1
:1040A000424AD05D012800D08CE03549204608F016
:1040B00037F93449204608F033F93349204608F0EF
:1040C0002FF93249204608F02BF93149204608F0F3
:1040D00027F9364AD05D012801D000F089FC284933
:1040E000204608F01DF92749204608F019F926490D
:1040F000204608F015F92549204608F011F9244911
:10410000204608F00DF99EE02E9924982150882031
:104110002150E555E56622462398249BD050166829
:1041200030681C903068379CA04330606007401EA8
:10413000B1680140B160576E002F204615D0B468B9
:10414000B068400F1D49095C1D4A105CC00007F0B3
:1041500073FF21010446480F1849095C184A105C96
:10416000C00007F069FF249B104A682150526A2062
:1041700014522A9815541C9830602E98D05024E080
:10418000CCD0000842CC000881C900082CC9000826
:1041900040CC000804FFFF070200000404000008F0
:1041A0000800000C8000001C400000181C100020BB
:1041B00000380140FFFF00FCA4110020E0D00008FF
:1041C000D8D00008576E1668249B2398D0503068CA
:1041D000379030680124A043306007204006B16862
:1041E0008143B160002F204615D0B768B068400FFA
:1041F000F849095CF84A105CC00007F01DFF04464E
:104200003801400FF349095CF34A105CC00007F025
:1042100013FF249BF14A682150526A2014523798A8
:1042200030602E9CD4502A9F2398D050D5553068AA
:1042300031681F461346012291433160510788437C
:104240003060DC515D66349EE54C01203090206684
:104250000721A164329FE76425656565A56522464F
:1042600040321D9802309080DE480346083B2364AC
:10427000527F002A0BD15C22A554DB4EB26B279BE8
:104280001A43B263B26B349E1A403D923D9A5D224E
:10429000A654C16001683943289B99430160856039
:1042A000016860239943016001682A9B994301607A
:1042B0003099A154CD482061459544954395429548
:1042C000207D00280A462AD165754E954D9501241A
:1042D0006007C54BD96B0143D963D96B0140389155
:1042E0003898586B20435863586B204038904C9551
:1042F00030204A90389803264B964AA922981746B0
:1043000006F026F93A46BA4B9868BA490840B10314
:10431000349E014399606004B7490860B04C26752B
:10432000256222753D953E953F95409541953DA866
:10433000294605F0EBFD002814D00026AF49304691
:1043400007F0EEFFAE49304607F0EAFFAD493046D0
:1043500007F0E6FFAC49304607F0E2FFAB493046D4
:1043600007F0DEFF3DA81021169105F0CFFD0028D3
:1043700014D00026A149304607F0D2FFA0493046AC
:1043800007F0CEFF9F49304607F0CAFF9E493046EE
:1043900007F0C6FF9D49304607F0C2FF9C489D4F7D
:1043A0009D4A9E49491E84C0056041608560C56084
:1043B0000561083806F038FB002814D000268F4924
:1043C000304607F0ADFF8E49304607F0A9FF8D4912
:1043D000304607F0A5FF8C49304607F0A1FF8B4916
:1043E000304607F09DFF8E488E4A8F49A6C0056073
:1043F00045608560103806F017FB002814D00026B1
:104400007E49304607F08CFF7D49304607F088FF33
:104410007C49304607F084FF7B49304607F080FF37
:104420007A49304607F07CFF8048856163228049E5
:10443000A6C00560103806F0F7FA002814D0002650
:104440006E49304607F06CFF6D49304607F068FF53
:104450006C49304607F064FF6B49304607F060FF57
:104460006A49304607F05CFFF2488561F924F24959
:10447000B2C0103806F0D8FA002814D000265F49E0
:10448000304607F04DFF5E49304607F049FF5D4971
:10449000304607F045FF5C49304607F041FF5B4975
:1044A000304607F03DFF3598E249085C0128EB4AA9
:1044B00015D100265149304607F032FF50493046A9
:1044C00007F02EFF4F49304607F02AFF4E4930468D
:1044D00007F026FF4D49304607F022FF25E03D203A
:1044E000349B0B5409684B68914201D1DC4A13405C
:1044F000702293438A684B60DA4B994207DC309B09
:104500009B07994209D0D84B994206D008E0D74B77
:10451000994202D0D14B994202D12A9B9A438A6098
:104520003599C44A555430991154D14EB561D1488A
:10453000B1C6103E304606F077FA002815D00026A6
:104540002E49304607F0ECFE2D49304607F0E8FED4
:104550002C49304607F0E4FE2B49304607F0E0FED8
:104560002A493046C24E07F0DBFE3598305C012800
:1045700015D100262149304607F0D2FE20493046A9
:1045800007F0CEFE1F49304607F0CAFE1E493046EE
:1045900007F0C6FE1D49304607F0C2FE56E03D203A
:1045A0003499315431684B68AC4A914201D1AC4ADC
:1045B00013402A9C702293438A684B60A94B99420E
:1045C00038DC309B9B0799423AD0A74B994237D0B1
:1045D00038E0C046E0D00008D8D000081C10002009
:1045E000C007002008300240001002400074004064
:1045F00008E400E0FF00FFFF00E100E0CCD000088D
:1046000042CC000881C900082CC9000840CC000831
:1046100014140020FFF9000000480140102700009A
:10462000601400205FEA000000440140AC14002048
:10463000002000408D4B994202D0884B994201D115
:10464000A2438A6035997554309931548A4FBD61BF
:104650002698401C209922C73D607860BD60083FC5
:10466000384606F0E1F9002814D000268349304688
:1046700007F056FE8249304607F052FE8149304627
:1046800007F04EFE8049304607F04AFE7F4930462B
:1046900007F046FE359C385D01282CD1002677496D
:1046A000304607F03DFE7649304607F039FE754941
:1046B000304607F035FE7449304607F031FE734945
:1046C000304607F02DFE385D01281FD16B4930467A
:1046D00007F026FE6A49304607F022FE6949304657
:1046E00007F01EFE6849304607F01AFE674930465B
:1046F00007F016FE30E03D21349C7C543868826817
:10470000634B13408360309A7A5401E03868349CDC
:104710003D217C544368514A904201D1504A134094
:1047200070229343826843604E4B984207DC309B73
:104730009B07984209D04C4B984206D008E04B4B5F
:10474000984202D0454B984202D12A9B9A438260FC
:1047500035983D54309878544E4C20460830852189
:104760004900199107F0F0FC4B4821C43D21785CC9
:10477000012820910DD102207854386839498842A7
:104780001DDC0121890788421FD0374988421CD08F
:1047900024E000253949284607F0C2FD384928465B
:1047A00007F0BEFD3749284607F0BAFD3B492846C9
:1047B00007F0B6FD3549284607F0B2FD12E02B4957
:1047C000884202D02549884208D182683449114084
:1047D000062907D001221204914203D00168012268
:1047E0000A4302602F4907F04FF900252E49284659
:1047F00007F096FD2249284607F092FD21492846F8
:1048000007F08EFD2949284607F08AFD1F492846F2
:1048100007F086FD2798411E254C20681891084016
:1048200024494018112814D8234E04A1085C4000E4
:104830008744C04630130020001400400D0F0F0FB6
:104840000F0F0F0F0F0F110F0F0F0F0F4A4B1B4EB4
:104850003BE01B4E39E01B4E37E0C046002C0140C8
:104860008FFF0FFFFF2B014000040040004001407C
:104870007C13002000100040C8130020CCD000089A
:1048800042CC000881C900082CC9000840CC0008AF
:104890008800CEFF600E0020C900010047CC000850
:1048A000070001005CCC0008BCD0000861CC000807
:1048B00000580140AAFBFFFF84C90008C8C90008CE
:1048C0003DC40008A6C900084C4E4D49284607F0D3
:1048D00027FD4C4F2846394607F022FD4A49284615
:1048E00007F01EFD2846314607F01AFD47492846C5
:1048F00007F016FD2068030C45493A4607F0C4F856
:104900002B9C2246383A434907F0BEF82246123A19
:10491000414907F0B9F84149B52207F0B5F8404ED2
:10492000B0688006400F21D0B068339C2040082832
:104930003C4A21D0B0682040102847D1F06829991E
:104940000840032800D0384AF0684006400F411C58
:10495000104607F071FBF1684904490E4843F168BD
:10496000490F491C07F068FB024605E030688004E7
:10497000400F2D4AC240339C2C4907F085F8B0689F
:104980008006400F0ED0B068204008280BD0B068D9
:104990002040102826D1F0682999084003284FD0DC
:1049A000214851E03068174C2149204604F0FAFABA
:1049B0002049204604F0F6FABFF34F8F1E49143900
:1049C0001E480860BFF34F8F00BFFDE7B06820406E
:1049D0002028219AD0D0B0682040182800D1A6E223
:1049E0002A46C9E7B06820402028DCD0B068DAE762
:1049F00016682E9C249BFFF717FCC046EAC90008E6
:104A0000BCD0000842CC000881C9000840CC000896
:104A100074CE00080CCA000890CE000842CA0008F4
:104A20000010024000127A000024F40072CC00084A
:104A3000C4CE000861C4000820ED00E00400FA05BF
:104A4000004801E000127A00F1684906490F491C4C
:104A500007F0F2FAF1684904490E4843F168490F3A
:104A6000491C07F0E9FAF84988429CD9F74C30987C
:104A7000A0603498A0601F9BA360F54E306A316A35
:104A80000A1A369917398A420BD2326A121A8A42A6
:104A900007D2326A121A8A4203D2326A121A8A4240
:104AA000EDD33098A0613498A061A361306A2C9B4B
:104AB0002A9D316A0A1A1946A7318A420BD2326AF4
:104AC000121A8A4207D2326A121A8A4203D2326A10
:104AD000121A8A42EDD32399DE4F785CDE4C183CE3
:104AE0000128206800D133E23794309C7C54252380
:104AF0000A46F95C012900D027E205933499F9545C
:104B00000021F96339680A68A2430A60BA6CFB6C39
:104B100053603A6D002A04D07A6DCE4B9B6D536082
:104B2000CC4F3A6C1C2301931A40309B9340CB4DE1
:104B30002A681A432A6030224A60BB68C84A102B90
:104B4000154600D005468D60102B00D01046C86079
:104B50000868309A104308600025C249284607F0CB
:104B6000DFFBC149284607F0DBFBC049284607F0B8
:104B7000D7FBBF49284607F0D3FBBE49284607F0BC
:104B8000CFFB0598B349085C022800D0F6E108681D
:104B90000068800600D5F8E10C6C01980440349858
:104BA000A040326AAD490B1F1E68064200D110E2D8
:104BB000A84C216D00290DD0626DA36D166833429B
:104BC00008D00E681E9F3E430E605360E16B369A1C
:104BD0001143E163A16CE26C0B681A42234604D0D6
:104BE0004A60D96B259A1143D96323995D549B4A36
:104BF000116808431060059830991954994928465E
:104C000007F08EFB9849284607F08AFB974928460B
:104C100007F086FB9849284607F082FB954928460D
:104C200007F07EFB8E483799086094480078652825
:104C3000934F2ED09349284607F072FB8A492846A5
:104C400007F06EFB8949284607F06AFB8E49284623
:104C500007F066FB8749284607F062FB8B488C49C2
:104C60000A4658C858C258C858C258C858C26520C1
:104C7000239A88543398C862886A401C886204F07A
:104C800061FB84488562C56205634563058704F05E
:104C9000C3FC04F0E9FB002814D000267E4930460E
:104CA00007F03EFB7049304607F03AFB6F4930464B
:104CB00007F036FB7949304607F032FB6D49304644
:104CC00007F02EFB764A1078282372493793C85490
:104CD0000B4628335078587090789870D078D870F8
:104CE000107918715079587190799871D079D8717C
:104CF000107A1872507A5872907A9872D07AD87264
:104D0000107B1873507B5873907B9873D07BD8734B
:104D1000107C1874507C5874907C9874D07CD87433
:104D2000107D1875507D5875907D9875D07DD8751B
:104D30008120420058885B4C0892A052088D412186
:104D40008A0099880C92A15211210A01D9880B92EC
:104D5000A1528321029149001A89625221210491B2
:104D6000CA0059890A92A1529989199AA1524321DC
:104D70008A00D9891A92A15230990902401C6052C6
:104D800087200D9040000793198A21524648339995
:104D90002F9A425446203290205A4A210E91615A4D
:104DA000414342480164E18F6E20484364211C91D5
:104DB00007F042F912996052E18B0804349E0BD03F
:104DC0000846309A1040012900D052E100282C9A60
:104DD0001F4B2B4F00D0A7E1608B6F28309900D07C
:104DE0003146652800D10021E08A228B1204101878
:104DF00004F0F8F85426B85D0128309600D1DCE1C3
:104E00000121B95538680246083283685B0700D52E
:104E1000B3E1146802231568ED0700D1EBE01C40F4
:104E200000D0E8E01468139D2C40012C00D0BBE1B9
:104E300084681F4D2C401C438460299C0460044CF2
:104E4000246A8568BAE0C046FF8FD0031004005082
:104E5000A41100207812002020ED00E004000240A0
:104E600000070020BCD0000842CC000881C900081F
:104E700053C7000840CC000810CF000824F00108F8
:104E800014120020C4D00008DCCE00088CC3000837
:104E9000C0060020C0070020CCD0000883CC00084A
:104EA00000F80108600E002028110020E405002011
:104EB000E8FFFF7F28688004410FF948C840359C0F
:104EC000A96889092140F74A51581F220A40D04059
:104ED000F54988644424F5490F5D002F01D13D4612
:104EE00001E0F34D1835349907F0A6F8401EF1495A
:104EF000884201D9FEF773FBEF494860EF4A10681A
:104F0000EC4B1840249B18431060002088600E6012
:104F1000002F01D1FEF763FB11460868F74A1040E5
:104F200028430860F3482F990155FEF76DFB179849
:104F3000020221E5A868104020282198C0D0A86866
:104F4000104018281ED00020BAE70020B854FD6396
:104F50000024EB49204607F0E3F9EA49204607F030
:104F6000DFF9E949204607F0DBF9E849204607F078
:104F7000D7F9E749204607F0D3F9FEE723980D5407
:104F80001F9803E0179800029AE71E98C863002450
:104F9000DB49204607F0C4F9DA49204607F0C0F99A
:104FA000D949204607F0BCF9DA49204607F0B8F99C
:104FB000D749204607F0B4F9FEE71568ED071AD087
:104FC000D54D2D6A2D1B032DF7D31568ED07F4D0B1
:104FD000EAE00826A6401F683E4200D0FCE0CE4929
:104FE0000F6ABF1A369918398F4200D905E119683E
:104FF0000142F0D0DCE5B955C84C641CBD6D2540BC
:105000000D43BD6500253D9514681668F6072F9E73
:10501000349500D1FDE01C4000D0FAE01468139DE7
:105020002C40012C1BD18468B34D2C401C43846060
:10503000299C0460B84C246A8668F6072F9E349D2C
:1050400000D1E6E0B44D03E01668F60700D1DEE0DB
:105050002E6A361B032EF7D31668F607F4D0BC6D04
:10506000169D2C43BC65FC6D0C43FC65349D2E469F
:10507000CFE0109FFE370F402C9B04E0AD1CBD42DB
:10508000349E00D1A2E6A6498E60A34E316A326AF0
:10509000521A9A420BD2326A521A9A4207D2326A92
:1050A000521A9A4203D2326A521A9A42EFD39C4958
:1050B000349A8A61316A326A521A9A420BD2326A3F
:1050C000521A9A4207D2326A521A9A4203D2326A6A
:1050D000521A9A42EFD39249349A8A60316A326AFC
:1050E000521A9A420BD2326A521A9A4207D2326A42
:1050F000521A9A4203D2326A521A9A42EFD388491C
:10510000349A8A61316A326A521A9A42B6D2326A43
:10511000521A9A42B2D2326A521A9A42AED2326AC3
:10512000521A9A42EFD3A9E77D4DAE60186A196A08
:10513000091A91420BD2196A091A914207D2196AC7
:10514000091A914203D2196A091A9142EFD3AE614A
:10515000186A196A091A914200D33DE6196A091AB8
:10516000914200D338E6196A091A914200D333E616
:10517000196A091A9142ECD32EE613689B0705D4ED
:1051800013685D4C2340169C23431360624B1B6ADB
:105190001468640700D43CE65F4C246AE41A032CCC
:1051A000F6D314686407F3D50020B855B86D169A85
:1051B0001043B865F86D0843F86500255049284646
:1051C00007F0AEF84F49284607F0AAF84E4928469E
:1051D00007F0A6F85349C1E000202399524A23461C
:1051E00014465054012002469A40504B196811430E
:1051F0001960E06305996054C9E6002023994A4A82
:1052000050542E98D063012005995054BFE62F9E2C
:10521000349D1468E407BC6D3FD1404D2C402E9363
:105220001C43BC65C468C768299B9F43C760324F55
:10523000183785683D4385601C403D4F1568002D3B
:105240003ED53D9D6D1C3D953D9DBD421AD81568CE
:10525000002D35D53D9D6D1C3D953D9DBD4211D820
:105260001568002D2CD53D9D6D1C3D953D9DBD4285
:1052700008D81568002D23D53D9D6D1C3D953D9D9D
:10528000BD42DBD92B493098349A0A54886D169A5E
:1052900010432E9A9043886552E016990C4318E00B
:1052A0000024F400B0C30008E40500202811002009
:1052B000E8FFFF7FFFFFFF0010E000E020ED00E0CF
:1052C000C2682243C2601B4FBC6D0C432E998C43B5
:1052D000349D30997D54BC65002E31D0B4214058A6
:1052E000129908403F3000901349144A054B06F0CC
:1052F000CBFB3AE028110020E8FFFF7FFFFFFF0013
:10530000CCD0000842CC000881C9000882CA00083D
:1053100040CC0008C0CA0008A4110020FDFEFFFF19
:1053200010040050D1CC0008781200200400024084
:10533000FFF1020014120020B0CC000808CF0008D2
:105340000025F649284606F0EBFFF549284606F009
:10535000E7FFF449284606F0E3FFF349284606F044
:10536000DFFFF249284606F0DBFFF1480069836B56
:1053700015990B40846BEF49E94D2A4606F084FBF2
:10538000E002C30EEC492A4606F07EFB01263046B9
:1053900002F0F0FB04F0B2F9002814D00025DF4938
:1053A000284606F0BDFFDE49284606F0B9FFDD4974
:1053B000284606F0B5FFE149284606F0B1FFDB4973
:1053C000284606F0ADFFDE4A50681F9988435060BA
:1053D000D749487D012802D10869DA4D25E0084601
:1053E00002210175006902683243026002683E23AF
:1053F0001340022BD34D02D1426832434260CC4A63
:1054000016751175D04AD21F036813430360159AAD
:105410005204036813407204934202D142680A4363
:1054200042600021C24A5175167500223D923D909E
:105430003D9908313D913D990A603D923D903D98DE
:1054400014303D903D981746026028681E99084226
:1054500008D028682599084204D02868369908425F
:1054600000D0A5E028681E99084208D1286825992F
:10547000084204D028683699084200D0E5E0286840
:105480001E99084208D028682599084204D1286846
:105490003699084200D0B2E028681E99084208D127
:1054A00028682599084204D128683699084200D016
:1054B00005E128681E9908421BD0286825990842F2
:1054C00017D028683699084213D12C6800259F49C7
:1054D000284606F025FF9249284606F021FF91490B
:1054E000284606F01DFF2B98044200D013E198498E
:1054F00035E028681E9908421FD12868259908427E
:105500001BD028683699084217D128682B99084281
:10551000904C01D002F0B6FA8F4803F023FD8F487B
:105520008F49904A904B914D2B656A65A965E86556
:105530008F4868600D22002656E12C6800258349BB
:10554000284606F0EDFE7649284606F0E9FE754944
:10555000284606F0E5FE2B98044214D185492846DA
:1055600006F0DEFE7149284606F0DAFE7B487C49EB
:105570007C4A7D4B7D4C23656265A165E0657C4876
:1055800060602D9A2FE17C49284606F0C9FE6749E4
:10559000284606F0C5FE71487149724A724B734C39
:1055A00023656265A165E0657448606004221AE1C4
:1055B0002C6800256549284606F0B2FE5849284661
:1055C00006F0AEFE5749284606F0AAFE2B98044284
:1055D00061D16B49284606F0A3FE5449284606F0DF
:1055E0009FFE68486849694A694B604C6360226560
:1055F0006165A065E065574C524D289AF5E02C682E
:1056000000265249304606F08BFE4549304606F0EA
:1056100087FE4449304606F083FE2B98044265D14C
:105620005C49304606F07CFE4049304606F078FE84
:1056300054485549554A564B4C4C63602265616548
:10564000A065E0650A22434CCFE02C6800253F4965
:10565000284606F065FE3249284606F061FE3149CB
:10566000284606F05DFE2B98044200D0A8E04A4987
:10567000284606F055FE2D49284606F051FE4148C1
:105680004649474A474B394C636022656165A065CE
:10569000E0650922A7E04449284606F041FE234977
:1056A000284606F03DFE37484049384A404B2F4CCB
:1056B000636022656165A065E0652A4693E028681D
:1056C0002B99084201D002F0AFF93A4803F04AFCA6
:1056D0002C483249324A334B244C63602265616561
:1056E000A065E0650B2200261A4C7EE03249304668
:1056F00006F016FE0D49304606F012FE21482B49F1
:10570000224A2B4B194C636022656165A065E065F8
:105710000222104C69E0294936E7C046CCD0000887
:1057200042CC000881C900083CC7000840CC0008F2
:10573000C0070020E2CC00080FCD000864CA0008B2
:10574000040002401004005007000100BCD0000813
:105750009ECB0008600E0020C8CB0008C98A000854
:10576000598A0008E989000889890008A4110020E5
:10577000F988000840CF000871CD0008358B00087B
:10578000F6CA0008010000200D850008C984000841
:105790004D8400084ACB000820CB00086187000830
:1057A0001D870008AD86000886C70008E58500084B
:1057B0006985000874CB0008DCC7000832C80008FF
:1057C000D049284606F0ACFDCF49284606F0A8FD92
:1057D000CE48CF49CF4AD04BD04C6360226561653B
:1057E000A065E0653246CE4CCE4D6285CE4806704F
:1057F00028682799084207D1CC4E2F9837997054C2
:1058000010321346628503E01346C84E379837546A
:105810002868119D284205D12F981B997054203378
:10582000638501E01B9837541E9804F06DFF25989E
:1058300004F06AFF369804F067FF2B9804F064FFC9
:10584000279804F061FF284604F05EFF319804F0C9
:105850005BFF219804F058FFB549AC4AAF4802609D
:1058600032657165B265F265B34BB24818670F20B7
:1058700080040F902998800506900120249040070D
:105880000390FA4D319713E010971746259AF84880
:105890000260BFF34F8FBFF36F8FEA2000212152C8
:1058A000F4485866F4480260F448B0653197109F98
:1058B00010979A4F18E002680A4302603398265402
:1058C000974C1A99605A401C60522798E849086022
:1058D000BFF34F8FBFF36F8F904F396A319881427A
:1058E000924E01D001F094FA386AF066F06EB16E13
:1058F000401A0228E24F49D3F06EB066608F196EED
:105900004018E821605201B22C981C304843FC49F1
:1059100006F072FBD821625E736E9A1A8018B53851
:10592000C217920C8218921362527066EA20235AB0
:10593000002B22D0347E002C21D0022B784C00D0BA
:1059400045E21104EF4A8A42C74B1FDD317A002934
:105950001CD1259BC6490B60BFF34F8FBFF36F8FE0
:10596000E949096900228A604A6122526748BE49B2
:105970004866C1480360BC4B49E2002004E00020B7
:10598000674C605270662F983076B74B387D002890
:1059900000D13FE14520C00034903858052800D29E
:1059A00030E127230146F85C28902498C7432E91C4
:1059B000881E2B900740D548461C002002E0801C22
:1059C000874274D0CD490C18E15C71408AB2560808
:1059D000C90719D06E407208F10718D15608D107CF
:1059E00019D06E407208F10718D15608D10719D0A6
:1059F0006E407208F10718D15108D20719D06940DA
:105A00004E08C90718D118E07208F107E6D06A40BD
:105A10005608D107E5D17208F107E6D06A4056086A
:105A2000D107E5D17208F107E6D06A405108D207E4
:105A3000E5D14E08C90700D06E403799625C7240CC
:105A40005108D20719D069404A08C90718D151082E
:105A5000D20719D069404A08C90718D15108D2079E
:105A600019D069404A08C90718D15108D20719D07E
:105A700069404E08C907A2D017E04A08C907E6D016
:105A80006A405108D207E5D14A08C907E6D06A4002
:105A90005108D207E5D14A08C907E6D06A40510843
:105AA000D207E5D14E08C90789D06E4087E72E9806
:105AB000C00702D11A4C914F5AE09049C8190F46BD
:105AC000C05C4640B0B24008F10737D0684041089A
:105AD000C007134C36D14808C90737D06840410881
:105AE000C00736D14808C90737D068404108C00709
:105AF00036D14808C90737D068404608C00736D1B4
:105B000036E0C046B1C7000840CC000801000020C4
:105B1000318800081D870008BD870008A4110020F7
:105B2000600E002010040050E40500202811002021
:105B3000C17C0008057D0008AC1000204108C007AA
:105B4000734CC8D069404808C907C7D14108C0078D
:105B5000C8D069404808C907C7D14108C007C8D0A4
:105B600069404808C907C7D14608C00700D06E4041
:105B70002E980246401C43424341384627302B9919
:105B8000415C1218521E127812025118B2B29142A0
:105B90002F9900D1194600295E4E334B32D122464F
:105BA000E18B289C2E910B1B59425941002C2F9BB5
:105BB00000D00B46012B2C4B144623D1317B0029FE
:105BC00028D11D9E28362899B9558B21890000239C
:105BD00011917B5037997C5C102C2B9600D17EE381
:105BE000062C00D187E3032C00D091E328990029EB
:105BF00000D1DBE32E9A8A4200D1D7E30B20862224
:105C000000F086FE002034997850387588202221D3
:105C1000414A11504E203490305A3099615A081A36
:105C20004142414152202152329831523598305CE4
:105C3000012801D000F023FC2621208C002801D16E
:105C400000F01FFC795C002901D000F01AFC3349F8
:105C5000884200DDA9E0411E1D2900D971E38800BA
:105C600008A108588746C046AC10002001A00000DB
:105C700080E100E00500002000E100E0557F000821
:105C8000240C0020215D00084B5E0008695E0008BE
:105C90004F630008A95F00084F6300084F630008C6
:105CA0004F6300084F630008616000084F630008FD
:105CB0004F6300084F6300084F6300084F630008FC
:105CC0004F6300084F6300084F6300084F630008EC
:105CD000C16000084F6300084F6300084F6300086D
:105CE0004F6300084F6300084F6300084F630008CC
:105CF0004F6300084F6300084D610008240C00202A
:105D0000FF0F00000000C4FFC0070020FEFF0000DE
:105D1000600E0020281100201C1000204F4F0000B2
:105D2000608BE94B9880A08BD880E08B1881208D08
:105D30005881608F9881A08F5882E08F988242208E
:105D4000205AD882E08A218B090408181860442060
:105D5000205A6521239A995418833398D86232982F
:105D6000205A5883A06CD8615620205A18844C20A1
:105D7000205AD8813498205A1882986A401C986218
:105D800003F0E0FA002800D190E200263046CF4927
:105D900006F0C6FA3046CE4906F0C2FA3046CD4982
:105DA00006F0BEFA3046CC497AE2CC49884238DC6B
:105DB000CB49884200D11BE2CA49884200D11AE28D
:105DC000C949884200D0C2E2C848186757E3032B8C
:105DD000C74B00D0DAE511040F9A914200DCD5E5FB
:105DE000317A002900D0D1E5259BC2490B60BFF371
:105DF0004F8FBFF36F8FC049096900228A604A61E3
:105E00002252BE48BA494866BD480360B84B2F9A33
:105E10003398325487204000215A491C2152327253
:105E2000B4E5B849884200D1EDE1B749884200D1D4
:105E3000F1E1B649884200D089E2F06DAF4988426D
:105E400000D01CE3B248F06519E3608B6F2800D1E5
:105E500067E2652800D06CE2E08A218B090408180B
:105E6000002103F0BFF809E3974E3046A9491CC949
:105E70001CC01CC91CC01CC91CC0652023997054BF
:105E80003398F062B06A401CB06203F05BFA0028FD
:105E900014D0002630468D4906F042FA30468C492F
:105EA00006F03EFA30468B4906F03AFA30469A49F7
:105EB00006F036FA3046994906F032FA00208E494B
:105EC00008878862C8620863486303F0A5FB03F093
:105ED000CBFA0028924C14D0002630467B4906F0BD
:105EE0001FFA30467A4906F01BFA3046794906F027
:105EF00017FA30468B4906F013FA3046874906F008
:105F00000FFA894A10787C49379BC8545078079B10
:105F1000587090789870D078D8701079187150793E
:105F2000587190799871D079D871107A1872507A26
:105F30005872907A9872D07AD872107B1873507B0E
:105F40005873907B9873D07BD873107C1874507CF6
:105F50005874907C9874D07CD874107D1875507DDE
:105F60005875907D9875D07DD87501200002098DF7
:105F7000215258880899605298880C996052D888A4
:105F80000B996052832040001989215258890A993F
:105F90006052988919996052D8891A99605287205D
:105FA0004000198A215269E2002630465F4906F016
:105FB000B7F93046464906F0B3F93046454906F090
:105FC000AFF930465A4906F0ABF93046594E5349BD
:105FD00006F0A6F93498305A3099615A81423AD184
:105FE000608B394B9880A08BD880E08B1881208DF6
:105FF0005881608F9881A08F5882E08F98824220CC
:10600000205AD882E08A218B09040818186044209D
:10601000205A6521239A995418833398D86232986C
:10602000205A5883A06CD86156243D48005B1884E0
:106030004C203B49085AD8813948349FC05B1882AC
:10604000986A401C986203F07DF93548005B344C37
:10605000F05330996052411E8841502160520DE248
:10606000A08DC01E80B23449884200D307E2379821
:10607000305C002800D102E23048006A1863304AE0
:1060800011682698086100204862209BD25C012A92
:1060900001D000F0ABFC0222294B209FDA55CB68DF
:1060A00001221343CB60274B994201DD00F08CFCA9
:1060B0009307994201D100F08DFC234B00F088FC3E
:1060C000002001F057FDD9E1C0060020CCD0000827
:1060D00042CC000881C9000810CC00086D9D00006A
:1060E000504F0000F9750000C5760000057D0008DE
:1060F000AC10002080E100E0C0070020010000207B
:1061000000E100E06E9D0000E3C4000058EC0000D8
:10611000C17E00088CC300084EC9000840CC0008AE
:10612000600E002083CC000800F80108BCD00008F5
:1061300037C9000828110020FEFF0000A41100202C
:106140007C130020FF2B014000040040E148016A5D
:10615000A08DC01E80B2E04A904200D38FE1186B40
:10616000081A369A183A904200D888E1DB488068CD
:10617000081ADB4A904200D881E1D848406C081ADE
:10618000904200D87BE1D7480268D368012083435E
:10619000D360136AD44F3B4208D1369B4433146A10
:1061A0001C42D24C02D1136883431360CD4A209F16
:1061B000D055CF4A1163CF4B1968269A0A61002245
:1061C0004A62DA5D012A01D000F019FE0222DA5596
:1061D000CA680243CA60C84A914201DD00F0FEFD70
:1061E0008207914201D100F0FFFDC44A00F0FAFDA0
:1061F000C348186743E1F06DC149884200D03EE1D1
:10620000C048F0653BE1F06DBD49884200D036E101
:10621000BD48F06533E1608BBC4B9880A08BD88083
:10622000E08B1881208D5881608F9881A08F5882D3
:10623000E08F98824220205AD882E08A218B09047C
:10624000081818604420205A6521239A995418830D
:106250003398D8623298205A5883A06CD86156205F
:10626000205A18844C20205AD8813498205A1882F9
:10627000A0681863986A401C986203F063F80028CD
:1062800014D000263046A24906F04AF83046A1490B
:1062900006F046F83046A04906F042F830469F49DD
:1062A00006F03EF830469E4906F03AF803F0DCF876
:1062B00000288F4B00D1E2E000263046944906F0DA
:1062C0002FF83046934906F02BF83046924906F0F5
:1062D00027F83046934906F023F83046CBE028995A
:1062E000002970D02E9A8A426DD003230B22862477
:1062F000249800F01AFC2899002974D02E9A8A421A
:1063000071D00598C0008621395402200B23EBE29E
:10631000B819249981702A994C404470299B00F047
:1063200008FCE08A218B09040818012102F05AFEBA
:10633000A4E0E08A218B09040818022102F052FE31
:106340009CE017998900884201D101F05CFB764AF4
:1063500010682699016100274762209BD15C0129C2
:106360000DD10221D154C26801210A43C260624AA0
:1063700090425CDC8A0790425FD0604A5BE0002676
:106380003046634905F0CCFF3046624905F0C8FF4E
:106390003046614905F0C4FF3046644905F0C0FF4E
:1063A0003046634E5E4905F0BBFF51E04479017908
:1063B000090209190A467E3A7C26F643B24200D306
:1063C00096E20320A2E24279017909028F18394648
:1063D0007C397A23DE4303239024B14200D39CE22C
:1063E00024981A46A9E2C278817809028B18892B71
:1063F00000D373E28D2189007958C95C022903D149
:106400004721C90079580988002900D166E2059919
:10641000C900149C7C5259004379344C6354611870
:1064200000794870B9190871CA7013985CE2414A42
:10643000904202D0404A904207D182683F4B1A40B6
:10644000062A05D00B049A4202D002680A43026071
:106450003598375438463A4905F062FF38462D4999
:1064600005F05EFF38462C4905F05AFF384635499D
:1064700005F056FF38462A4905F052FF1C4B002014
:106480002084144F386A596B884201D1FFF725FAEE
:10649000586378692C4909694140BA680A40D34376
:1064A000BB60FC680C405C40FC604A4022405040AD
:1064B00078610240B969114302462D9B1A4045D0CC
:1064C0003B695B1E3B6143D11C9B3B61FB691343F2
:1064D000FB613DE0A4110020FEFF0000E405002068
:1064E000102700006014002011110000600E002031
:1064F000AC10002030130020FF2B014000040040AE
:1065000001000020C97D0008657D0008C00600204C
:10651000CCD0000842CC000881C900085CD000083B
:1065200040CC000883CC00081414002080D0000860
:106530002811002000400140002C0140070001000C
:10654000C4D0000852CE0008000C0050FC4A3A614A
:106550000B468343082213405940B961002BF94C84
:106560006AD000263046F84905F0DAFE3046F74991
:1065700005F0D6FE3046F64905F0D2FE3046F54924
:1065800005F0CEFE3046F44905F0CAFE396AA08D0A
:10659000C01E80B2F14A9042F14B01D3FFF79DF942
:1065A000186B081A369A183A904201D8FFF795F9F5
:1065B000EC488068081AEC4A904201D8FFF78DF940
:1065C000E848406C081A904201D8FFF786F9E7487E
:1065D0000268D36801208343D360136AE44C2342EA
:1065E00007D1369B4433146A1C4202D1136883439B
:1065F0001360DE4A209C1055D94A1163DD4B19689F
:10660000269A0A614E621A5D012ADB4C2F9E00D049
:1066100059E10222209FDA55CA680243CA60D74A6C
:10662000914200DD3EE18207914200D140E1D44A2F
:10663000914200D13CE143E1FB691C4694430B408D
:1066400013405940B961FC61002B43D0002630460D
:10665000BD4905F065FE3046BC4905F061FE304697
:10666000BB4905F05DFE3046C64905F059FE30468F
:10667000B94905F055FEB34CA08DC01E80B2B74994
:106680008842B74B01D3FFF728F9BB483799405CE4
:10669000002801D1FFF721F9386A1863BA4A106857
:1066A000269901614662209C115D012900D09BE082
:1066B00002211155C26801210A43C260AF4A9042CB
:1066C00000DD7EE08A07904200D180E0AC4A904233
:1066D0007DD086E00A468243042010404140B961E3
:1066E0000028984C9E4B01D1FFF7F7F80026304662
:1066F000954905F015FE3046944905F011FE3046E7
:10670000934905F00DFE3046A04905F009FE3046DC
:10671000914905F005FE924B186B396A081A2C9ABC
:10672000A632904201D8FFF7D8F890480268D368A3
:1067300001208343D360136A8D4F3B4208D1369BBF
:106740004433146A1C427F4C02D1136883431360A4
:10675000864A209F2E90D055A28D002A804C00D0D2
:106760002163784B9E85259A89490A60BFF34F8F34
:10677000BFF36F8FEA215E528649616686490A60DF
:10678000864B1968269A0A614E62854A7A48826564
:10679000844A854C1460854A0265DA5D012A2E9888
:1067A0006CD102227D4BDA55CA680243CA60734A33
:1067B000914252DC8207914255D0714A914252D0A7
:1067C00059E07B4A904202D07A4A904209D18268CD
:1067D000794B1A40624B062A06D00B049A42604B52
:1067E00002D002680A430260604A1068269901617B
:1067F0004662115D0129604C2F9E01D0FFF75EF8C3
:1068000002215A4A209BD154C26801210A43C26026
:106810005A4A904208DC8A079042514B0DD0584AA0
:1068200090420AD0FFF747F8614A90424C4B04D09F
:10683000604A904201D0FFF73EF882685E4B1A40F2
:10684000474B062A01D1FFF739F80B049A42444B13
:1068500001D1FFF733F8FFF72EF8554A914202D0E5
:10686000544A914207D18A68534B1A40062A05D0F0
:1068700003049A4202D00A6802430A604F48006843
:106880001E9901602599016027994D480160424891
:106890000160334B9E673848067206715E67294C6B
:1068A000FFF71AF8424A914202D0424A914207D178
:1068B0008A68414B1A40062A05D003049A4202D046
:1068C0000A6802430A60339826541E4C1A99605A8B
:1068D000401C6052334F224BFEF7FFFF0598C0006B
:1068E000862139540223184639188B55431C20E160
:1068F000C27880780002821810468A1811468A39B8
:106900008826F643B14200D3A9E00220029A2B9ECA
:10691000B91988704A70299B0BE1C178807828905A
:10692000000209914618BF1938468A388821C943A0
:10693000884200D3CCE002222498224F2B9EF4E020
:106940005F090000600E0020BCD0000842CC0008A7
:1069500081C90008F2CB000840CC0008FEFF00000F
:10696000AC100020E4050020102700006014002077
:10697000111100003013002028110020FF2B0140CE
:106980000004004088C800087C1300208CCF000859
:1069900080E100E00500002000E100E0AC140020F0
:1069A000498D0008A4110020F18B0008CD83000858
:1069B00000400140002C014007000100141200209B
:1069C00080E200E0240C0020F44B994202D0F44B0A
:1069D000994208D18B68F34F3B40062B06D0140434
:1069E000A342F14C02D00B6813430B60EF4B1968C4
:1069F000269A0A6148622098185C012820D102205A
:106A0000EA4A209BD054CA6801200243CA60E84A7F
:106A1000914204DC8207914207D0E64A03E0DF4A54
:106A2000914202D0DE4A914207D18A68DD4B1A407A
:106A3000062A05D003049A4202D00A6802430A607B
:106A40002F98339970541A99605A401C60522798B5
:106A5000D9490860BFF34F8FBFF36F8F0EE52B99B5
:106A6000791864008C7003244C7004464100104671
:106A7000CD4A511809912E94F918099AD6187778A9
:106A8000952464000F552893D25C0F192E9C7A70C0
:106A9000611C814200D378E1F178B970B178F97066
:106AA000A11C814200D372E1717939713179797118
:106AB000E11C814200D36CE1F179B971B179F971CE
:106AC0000833241D8442BD4FD5D3DB1C2B9931E004
:106AD0007000B5490B184720C000B84C20582E90C4
:106AE0008D20800020582F3409E021781970611E14
:106AF000097859709B1CA41C761CBE4209D2815D8A
:106B00000029F7D00229F0D12E9909880029ECD16B
:106B1000F0E7AA4F2B9EB8190999C1702899817086
:106B20001699417000241F98149B381884558019B9
:106B3000427031461E46249886431A4602402E92E1
:106B40007A189F48441C304602E0921C801E72D086
:106B5000117861404C08C90719D06C406108E407FE
:106B600018D14C08C90719D06C406108E40718D146
:106B70004C08C90719D06C406108E40718D14F08C8
:106B8000C90719D06F407C08F90718D118E06108CF
:106B9000E407E6D069404C08C907E5D16108E4077D
:106BA000E6D069404C08C907E5D16108E407E6D0A2
:106BB00069404F08C907E5D17C08F90700D06C404F
:106BC000577867407908FC071AD069407B4F4C081A
:106BD000C90719D16108E4071AD069404C08C907F0
:106BE00019D16108E4071AD069404C08C90719D1C6
:106BF0006108E4071AD069404C08C907A5D018E01D
:106C00006E4F4C08C907E5D06C406108E407E4D139
:106C10004C08C907E5D06C406108E407E4D14C0892
:106C2000C907E5D06C406108E407E4D14C08C90706
:106C30008BD06C4089E72E98002802D1200A2F9E25
:106C40003DE0B8192B99405C4440A0B24008E107F0
:106C50001AD068404108C0072F9E19D14808C907BB
:106C60001AD068404108C00719D14808C9071AD08E
:106C700068404108C00719D14808C9071AD06840C0
:106C80004408C00719D119E04108C0072F9EE5D07C
:106C900069404808C907E4D14108C007E5D0694008
:106CA0004808C907E4D14108C007E5D06940480851
:106CB000C907E4D14408C00700D06C40200AF91885
:106CC0002B9A8C548918487026202D9939549B1C76
:106CD00011983B5098B24142414138680246803297
:106CE0005468202C344600D10C46002C44D18668D0
:106CF00027998E4202D1016900293DD011780129DE
:106D00003AD0014654314B80D4600B802B997918CE
:106D1000016504995160416E039B994216D12799F0
:106D20008E4203D101690029264900D026491470FA
:106D30004167EFF31081249A82F31088D20500682E
:106D400083681343836081F3108815E027998E428E
:106D500003D1016900291D4900D01D491470416704
:106D6000EFF31081249A82F31088006802682A9B4E
:106D70001A43026081F310880020349978503875E6
:106D8000144E094C144BFEF745FF5B1D02E0DB1D62
:106D900000E00933094F2B99CCE6C0460040014082
:106DA000002C014007000100600E0020601400204C
:106DB000FF2B01400004004080E100E0240C002093
:106DC000FEFF0000FDB30008C5C5000875B400084B
:106DD00031C6000828110020AC100020F44A91426E
:106DE00002D0F44A914207D18A68F34B1A40062A2E
:106DF00005D003049A4202D00A6802430A602F9821
:106E0000339970541A99605A401C6052FFF736FB50
:106E1000F06D2E918047306D8047706D80473868E7
:106E20008047B06D8047E54BE54A506840005060B0
:106E3000229909694904C90F401850602E9900D160
:106E40000DE1586D081A4E2800D208E15965DD4958
:106E5000DD4F3A46DD4B04F017FEDD49DD4A3B4687
:106E600004F012FED820225EDB4904F00DFED84962
:106E7000D84A3B4604F008FEFC20225ED74904F0C5
:106E800003FED349D34A3B4604F0FEFDEC20225ECC
:106E9000D34904F0F9FDCE49CE4A3B4604F0F4FD57
:106EA000CC20225ACF4904F0EFFDC949C94A3B46DC
:106EB00004F0EAFDD220225ACB4904F0E5FDC44992
:106EC000C44A3B4604F0E0FDCA20205A0028C74AC5
:106ED00000D0C74AC74904F0D7FDBD49BD4ABA4BE7
:106EE00004F0D2FDC820205A0028C04A00D0C04A71
:106EF000C14904F0C9FDB649B64C2246B24F3B46E3
:106F000004F0C2FDBD480069C26ABD4904F0BCFD81
:106F1000AF4922463B4604F0B7FDB8480069026B12
:106F2000B84904F0B1FDAA4922463B4604F0ACFD45
:106F3000EA20B54C205A0028B44A07D0012801D1D4
:106F4000B34A03E00228B34A00D0B34AB34904F07D
:106F50009BFD9F499F4A9C4F3B4604F095FDE220D4
:106F6000A94C205EAE494143CA0F89148A1826995C
:106F7000083951430818C1174840431AA94904F079
:106F800083FD9349934A3B4604F07EFD2046F62458
:106F9000005BC007A44F03D03946A44A04F074FD37
:106FA0003946A34A04F070FD89498A4A864B04F0A9
:106FB0006BFD9548005B800703D539469B4A04F07A
:106FC00063FD39469B4A04F05FFD8149814A7E4B4F
:106FD00004F05AFD8C48005B400703D53946934ABC
:106FE00004F052FD3946944A04F04EFD7849794A3E
:106FF000754B04F049FD8448005B000703D5394612
:107000008A4A04F041FD39468C4A04F03DFD70493E
:10701000704A6D4B04F038FD7B49085B0C468006D6
:1070200003D53946814A04F02FFD39467A4A04F0E7
:107030002BFD6749674A644B04F026FD80480069D0
:10704000C007804A04D039467F4A04F01DFD7F4ABC
:10705000394604F019FD7E4904F016FD574B3420E3
:10706000315C00290D9900D17A499A6B2E9FBA1A8A
:107070008A4200D8DBE32F993154CC246248005B6C
:10708000996D0E1AF017864373480E99405A71494C
:107090004843000B71494843714904F0CDFF474B09
:1070A0008019C108584A1153574A9F63986588B29E
:1070B000D021515A814202D21146D03105E0CE2171
:1070C000515A814202D91146CE310880D2244E480D
:1070D000005B3B4FF96B0E1AF01786435E483299FE
:1070E000405A5C494843000B5C4948435C4904F002
:1070F000A3FF80194109444A1153434CF86388B2F5
:107100005849884217D8584E317800291ED12F9CF3
:1071100033997454F6213C4A525A082313433A4A8D
:10712000535283214900384A525A521C364B5A5204
:107130003470354C0AE04D4988424B4E06D3F62157
:10714000625A08239A43625200213170D621615A53
:10715000814202D22146D63105E0D421615A8142D2
:1071600002D92146D431088044213B482B91405A12
:107170003F4948433F4940183F4904F03DFFE22161
:10718000625E0E4FFB6B9A1A3C4B9A181218293A02
:10719000D017C00E101840116052FA63224604B294
:1071A000E621515E8C426BDD1146E6316EE0C04651
:1071B00000400140002C014007000100AC100020FD
:1071C000E4050020BECD000808CF000842CC00082E
:1071D000ACCF0008A4CF0008B4CF0008C0CF00088F
:1071E000C3CD0008A3C80008AEC8000808CC00083A
:1071F000CCCF0008CCCD0008D5CD0008C0070020BA
:10720000B9C80008C4C80008600E0020CFC8000834
:10721000D2C80008D5C80008D8C800080ACC0008A1
:1072200067660000DECD0008DBC80008A0D00008BB
:10723000DEC80008E1C80008E4C80008E7C8000884
:10724000000C0050ECCF0008DCCF0008E4CF0008B1
:1072500040CC0008B80B0000A4110020A8DE0000FC
:10726000102700000F27000028110020E12E000049
:10727000140500000CE3F7FFEF060000FDFEFFFF22
:10728000E421515E8C4203DA1146E4310880EE4A73
:10729000118D8C4214DA4B204843642104F0CCFE5B
:1072A000EA4FA042E84C1DDD1B98305C002819D045
:1072B000F620215A0122914321520020307111E021
:1072C00030790028E04C0DD12F9B33983354F620B1
:1072D000215A01220A4322520899605A401C6052E6
:1072E0003371DA4FB86F401E414241414900F620E8
:1072F000225A26239A4351187A6F521E5342534101
:107300009A005118327A531E9A4152010A4322526E
:10731000D820235E002B06D4DC20215A8B420ADDC4
:107320002352CA4A14E0E021625A5842904209DDD1
:107330006052C64A0CE0DA20215A8B42C34A07DA6F
:10734000235205E0DE21625A9042C04A00DA6052C0
:10735000906EF8216052D06EFA216052906C116CE0
:10736000081A916E0918C817000F28910818011102
:107370004C203190205A8842119101DC0E1A00E015
:107380000026D06C516C081AD16E0C18E017000F53
:1073900020180711AC483499405AB842099301DCCF
:1073A000C01B3618AA487043AA4904F025FEFC21E8
:1073B000A54A5052A54828990164446411998164F2
:1073C000C7642C98A63034904643D18F144630467B
:1073D00004F012FEEC216052EA20205A9E4B196DF7
:1073E000002802D19D4A914207D1012802D19C4A2E
:1073F000914202D19B4A914200D01A659A4A116982
:1074000012699A4B1B785E425E414906C90F711A98
:107410004B1E9941CA238C4CE152D1B2C909711A51
:107420004A1E9141C822A152401E02280BD8099839
:107430000328864B2B9E0DDB01208D4988613498F3
:107440001865814A13E00120894988627E4A7F4B92
:107450002B9E0CE000287C4A09DC186D012801DB1A
:10746000401E1865002802D1012081498862905B86
:1074700048247949095B8142918F2B9119D0884228
:1074800017D9734A511E89B2884202D96E48825375
:1074900010467149085318994843114604F0CCFD31
:1074A0006949329A88520E9A895A41436F48016459
:1074B000664B654A105B684E0E99715A814214D032
:1074C0001E2802D8159860490853634E0E9C30530D
:1074D00068494843684904F0AFFD5B4A105332994C
:1074E000515A414361480164584B22980069C005D4
:1074F000C00FFE21505242203490105A3199715ED3
:10750000814214462E9F00D191E15C49309A895CFA
:1075100001294F4B2B9A08D19042014600D900E136
:107520001146904200D3FEE0FFE01F46012253487F
:1075300030992B92425401688A6852075CD44F48B4
:10754000036D1A4624325478022C2ED15478022C22
:1075500000D09DE01E6834680E20844334604848A3
:10756000871C586C046828973C40046030682B9F47
:10757000B8433060186C019C20408740414E306811
:1075800038433060986CDC6C44601E6D002E06D071
:107590003068289C20403060586D9B6D436000200F
:1075A00010702B9850702C4E294F4868169A9043B3
:1075B00048608B688868C007234C3DD00222134086
:1075C0003AD1886805230340012B00D08EE08868FB
:1075D0002D4B184010438860032008602B48026A36
:1075E0008868C00728D02948006A801A0328F7D382
:1075F0008868C007F4D079E08A68920705D48A6861
:1076000021480240169802438A602048026A8B682B
:107610005B0794D51D48036A9B1A032BF7D38B682D
:107620005B07F4D51548816D169A11438165C16DCC
:107630002B9A1143C16568E01148401C0F4A936DB5
:10764000034058325AE0C046600E0020AC100020C3
:10765000B80B0000FF0F000028110020CD830008A8
:10766000E98300080584000800080050E4050020B4
:10767000000C005000E2040040420F0014120020F1
:10768000FDFEFFFF04000240E8FFFF7FA411002081
:107690000420D863F64CA06D129B1843A06548687F
:1076A000169B98434860002010708B688868C0075C
:1076B000F04C26D00222134023D1886805230340D2
:1076C000012B13D18868EC4B1840104388600320CD
:1076D0000860EB48026A8868C00712D0E848006A70
:1076E000801A0328F7D38868C007F4D0E04B986D60
:1076F000169A104398651A465C32DB6D2B9803434B
:107700001360C8682B9A9043C8600020F949309AEA
:1077100088543498205AA28F3B469042014600D8A4
:10772000FEE6904201D3994205D9994200D3194609
:10773000349821520846319970520021319142917A
:10774000ED493F9106993E91CC493D9101244094E9
:10775000189948431F46194604F06EFC41903DA815
:1077600002F03EFA002814D000263046DA4904F030
:10777000D7FD3046D94904F0D3FD3046D84904F04E
:10778000CFFD3046D74904F0CBFD3046D64904F052
:10779000C7FD3DAE3473D9483F9006983E90EC4803
:1077A0003D9031984290D74C3498205A18994843CC
:1077B000394604F041FC4190304602F011FA0028AD
:1077C00014D000263046C44904F0AAFD3046C3490F
:1077D00004F0A6FD3046C24904F0A2FD3046C1497E
:1077E00004F09EFD3046C04904F09AFD01F086FF8A
:1077F000002814D000263046B74904F091FD3046E9
:10780000B64904F08DFD3046B54904F089FD304697
:10781000BE4904F085FD3046B34904F081FDB34A0A
:107820005068042188435060A84EC54B2E9F306E8F
:10783000381A1A283A4621D33266707C4000707498
:1078400022990969219A11420FD1012108437074CC
:10785000307D00282E9A11D12F993175307B002868
:1078600009D000203073B54807E000062E9A05D1F4
:107870000020307502E03173B6487065109FD01B50
:10788000B549884240D3002630469F4904F048FD60
:107890003046924904F044FD3046914904F040FDE1
:1078A0003046AE4904F03CFD30468F4904F038FDC7
:1078B0002E9AA34B85483399405C0128174623D163
:1078C0000120000220588E4988620C98205A888531
:1078D0000B98205AC88583204000205A08860A98B1
:1078E000205A48861998205A88861A98205AC8869D
:1078F00087204000205A088701F08EFE2E9A904B78
:107900007248339946541746A08D022815D0012895
:1079100031926E4E01D0FDF7CBFF3079012801D1B5
:10792000FDF7B2FF986F01283ED0307A01284AD087
:10793000586F012856D0FDF7BBFF644E3079002800
:107940002F9800D13078C00723D0307C00283192A6
:1079500001D0FDF7ADFF259A7A480260BFF34F8F43
:10796000BFF36F8FEA2000212152784858666048A3
:1079700002603079012801D17C48B0653078012857
:107980002E9901D17A48B0652F9830743191FDF766
:107990008FFF986F01280BD1307C0028319201D0E5
:1079A000FDF786FF2F9830746F48B065FDF780FFB4
:1079B000307A01280BD1307C0028319201D0FDF7BC
:1079C00077FF2F9830746748B065FDF771FF586FE7
:1079D00001280BD1307C0028319201D0FDF768FFDF
:1079E0002F9830745E48B065FDF762FF317C3948EE
:1079F0001346426818469047514B002030742E9829
:107A00003190FDF755FF3E480069002181604161DA
:107A1000EA202152BFF34F8F2D4914394A4808609C
:107A2000BFF34F8F00BFFDE700263749304604F013
:107A300077FC2A49304604F073FC2949304604F0AB
:107A40006FFC3749304604F06BFC2749304604F0A0
:107A500067FC2F482F49304A304B1E4C636022652B
:107A60006165A065E0650322264CFDF7BEFEC046B9
:107A700014120020600E0020E8FFFF7FFFFF1700B8
:107A8000A411002000262049304604F049FC134987
:107A9000304604F045FC1249304604F041FC2649CA
:107AA000304604F03DFC1049304604F039FC1D48D6
:107AB0001D491E4A1E4B074D2B656A65A965E86581
:107AC0001C4868600522FDF78FFEC0462811002083
:107AD00020ED00E0A4110020CCD0000842CC00082A
:107AE00081C900082CC9000840CC000804000240ED
:107AF00000E100E01412002004000008400000181B
:107B0000C0070020600E0020BCD0000864CA000836
:107B100001000020318800081D870008BD8700088B
:107B200007C80008C98A0008598A0008E9890008BE
:107B300089890008358B00085DC80008C17C0008F1
:107B4000AC10002080E100E00400FA0505000020F0
:107B5000FFFF2700397F0008C1D401003CCD000899
:107B6000E9810008FD80000815800008557F0008A5
:047B7000D9820008AE
:107B7400F0B582B03C4F396B3C4A146A01221302BF
:107B8400002806D1601A1946F431884201D802B09F
:107B9400F0BD37480168CD689543CD600D6A354E18
:107BA400354206D10D6A344E354202D10D689543F3
:107BB4000D6001933D214254304DA88D002800D022
:107BC4003C630020A88553022D4E3360BFF34F8FD2
:107BD400BFF36F8FEA26A8532A4D7D662A4D009382
:107BE4002B60D743294E35682F616862284B294F93
:107BF4009F65294F1D4C2760284F1F65775C012F17
:107C0400019B1FD102277754E9681143E960244995
:107C14008D4206DC91078D4209D024498D4206D05D
:107C24000DE020498D4202D01F498D4207D1AE6834
:107C34001F493140062905D01604B14202D02968F3
:107C4400114329601B4909680B60009B0B601103F9
:107C5400194A11600C4A1160034988670C4A107272
:107C64001071486702B0F0BDAC100020A4110020D0
:107C7400601400201111000044040000600E002074
:107C840080E100E00500002000E100E0AC140020E9
:107C940028110020498D0008F18B0008CD830008CD
:107CA400FF2B014000400140002C01400004004033
:0C7CB400070001001412002080E200E034
:107CC00070B50F4802780A494C690A4B1B6A1D1BA4
:107CD000094C002A03D0332D09D3103402E0074E9B
:107CE000B54204D9012525606A4002704B6170BD20
:107CF000AC100020A411002018040050B6030000AE
:047D00004C11002002
:107D040010480069002282604261EA200E490A524A
:107D14000E480F4A4266826F002A00D07047426FB5
:107D2400002A07D10D4A01231370112212018B5A24
:107D34005B1C8B52012141670648006A0649886032
:107D44007047C046C0070020600E0020AC10002021
:107D540001000020A4110020E4050020601100208F
:107D6400F0B581B000240F4F25463E6E3B6E0E49A0
:107D7400224603F087FE7519641C0C488442F4D132
:107D84000146284604F056F90949081A0949488762
:107D940002B2094903F076FE08480949C16501B0F9
:107DA400F0BDC046AC10002011C9000850C300004B
:107DB400FF070000600E00203DCE000828110020BF
:047DC400010000209A
:107DC800F0B581B000252D49284604F0A5FA2C49C4
:107DD800284604F0A1FA2B49284604F09DFA2A49BE
:107DE800284604F099FA2949284604F095FA284EBD
:107DF800376A306AC01B2749884224D22C4604E0DF
:107E0800306AC01B234988421DD2601B2249C96EB3
:107E18000C18E017000F2018051120492A4603F016
:107E28002FFE306A316A091A0129E9D8316A091A1C
:107E38000129E5D8316A091A0129E1D8316A091AF4
:107E48000229EFD3DCE71B4E708A2D1AACB26E20E4
:107E58006043642104F0ECF8B080758010486843F2
:107E6800104904F0C5F8308083B20F49224603F068
:107E780007FE0E480E49C16501B0F0BDBCD0000830
:107E880042CC000881C90008EAC8000840CC0008B4
:107E9800A411002060EA0000AC100020F4CF000814
:107EA800B80B0000FF0F000014D0000828110020B4
:087EB800010000209C0E0020D7
:107EC000F0B583B000252C462F461448866EC16E4F
:107ED0000291836EC06E009011492A4603F0D4FDD2
:107EE00034190298C7196D1C0E488542EDD105461C
:107EF0003846294604F0A0F806460E4F7880204602
:107F0000294604F099F8388082B2B3B2064903F0EA
:107F1000BBFD06480649C16503B0F0BDAC100020AA
:107F2000EBCD000850C3000018CE00082811002037
:087F300001000020AC0E00204E
:107F38000348044941650448012101607047C0466F
:0C7F480028110020010000201804005047
:107F540010B52A48026A2A494B68002B09D000222E
:107F64004A60016A2948426F002A0DD00021416706
:107F740010BD8B68022B2AD0012B10D0002BF0D11E
:107F8400214B08241C6011E0826F022A2AD0012AA6
:107F940011D0002AECD11C4A0223136012E00B68B2
:107FA400D31AC92BDDD3184B08241C610A608A68D4
:107FB400521C8A60D5E7026F8A1AC92AD8D3124A9A
:107FC400022313610167816F491C816710BD0B682F
:107FD400D31A0C4CA342C4D90A60002201234B607B
:107FE4008A60BEE7026F8A1A064B9A42C0D90167BB
:107FF400002101224267816710BDC046A411002000
:10800400AC100020C40900001804005028110020FE
:1080140030B582B06846C821018001AA1180518020
:108024003049418030494B683048026A012B0AD8F4
:108034008C68022C18D0012C08D0002C20D12C4B99
:1080440008241C600CE000224A6019E05B0001ACCB
:10805400E35A0C68141B9C4212D9254B08241C615A
:108064000A608A68521C0AE05C006D462C5B0D684D
:10807400551BA54204D90A6000225B1C4B608A6030
:108084001C494A6F006A012A0AD88B6F022B1BD045
:10809400012B09D0002B05D1154A022313600DE0F2
:1080A4000020486702B030BD520001AB9A5A0B6FF2
:1080B400C31A9342F6D90E4A022313610867886FE4
:1080C400401C886702B030BD53006C46E35A0C6F05
:1080D400041B9C42E6D908670020521C4A67886743
:1080E40002B030BDC4090000AC100020A41100206F
:0880F4001804005028110020BF
:1080FC0030B584B06846C821018002AA1180518035
:10810C00418091803049818030494B683048026A07
:10811C00022B0AD88C68022C18D0012C08D0002C09
:10812C0020D12C4B08241C600CE000224A6019E082
:10813C005B0002ACE35A0C68141B9C4212D9254B11
:10814C0008241C610A608A68521C0AE05C006D46B7
:10815C002C5B0D68551BA54204D90A6000225B1CE0
:10816C004B608A601C494A6F006A022A0AD88B6FDE
:10817C00022B1BD0012B09D0002B05D1154A022351
:10818C0013600DE00020486704B030BD520002AB14
:10819C009A5A0B6FC31A9342F6D90E4A02231361F3
:1081AC000867886F401C886704B030BD53006C466C
:1081BC00E35A0C6F041B9C42E6D908670020521C42
:1081CC004A67886704B030BDC4090000AC100020B9
:0C81DC00A41100201804005028110020FD
:1081E80030B584B06846C821018002AA1180518048
:1081F800418091808180D1803049C18030494B686D
:108208003048026A032B0AD88C68022C18D0012C3B
:1082180008D0002C20D12C4B08241C600CE0002234
:108228004A6019E05B0002ACE35A0C68141B9C42DC
:1082380012D9254B08241C610A608A68521C0AE07E
:108248005C006D462C5B0D68551BA54204D90A607D
:1082580000225B1C4B608A601C494A6F006A032A33
:108268000AD88B6F022B1BD0012B09D0002B05D10C
:10827800154A022313600DE00020486704B030BDA2
:10828800520002AB9A5A0B6FC31A9342F6D90E4AA0
:10829800022313610867886F401C886704B030BDEB
:1082A80053006C46E35A0C6F041B9C42E6D90867DE
:1082B8000020521C4A67886704B030BDC40900001A
:1082C800AC100020A4110020180400502811002030
:1082D80030B586B06846C821018003AA1180518054
:1082E800418091808180D180C18011813049018194
:1082F80030494B683048026A042B0AD88C68022C33
:1083080018D0012C08D0002C20D12C4B08241C603C
:108318000CE000224A6019E05B0003ACE35A0C68E9
:10832800141B9C4212D9254B08241C610A608A68D8
:10833800521C0AE05C006D462C5B0D68551BA5427B
:1083480004D90A6000225B1C4B608A601C494A6F92
:10835800006A042A0AD88B6F022B1BD0012B09D084
:10836800002B05D1154A022313600DE00020486751
:1083780006B030BD520003AB9A5A0B6FC31A934232
:10838800F6D90E4A022313610867886F401C886774
:1083980006B030BD53006C46E35A0C6F041B9C4278
:1083A800E6D908670020521C4A67886706B030BDC6
:1083B800C4090000AC100020A411002018040050CB
:0483C8002811002058
:1083CC000348044901650448042101607047C04614
:0C83DC002811002001000020280400509F
:1083E8000348044901650448042101607047C046F8
:0C83F80028110020010000201804005093
:1084040070B5104802780B490C690B4B1B6A1D1B95
:108414000A4C002A03D0332D0AD3103402E0084E4C
:10842400B54205D9042525600124624002700B6120
:1084340070BDC046AC100020A411002018040050E8
:08844400B603000048110020FE
:10844C0010B5002901D0022426E0154A516A431ABE
:10845C0014494C6AA34221D95062134800680A7827
:10846C00002A0AD0C0B2C409886AA0420BD0A0006E
:10847C00104A1018006D104A07E0FF228243D409FD
:10848C00886AA042F3D1094A0948A300D2584A622B
:10849C000849C918C86380470248846210BDC046A9
:1084AC00AC100020E40500201008005064C3000844
:0C84BC0001000020A41100205CC3000897
:1084C80001204102084A1160BFF34F8FBFF36F8F3D
:1084D8000B4A10800548064A42660648016006486D
:1084E800064901607047C04680E100E0AC100020FA
:1084F8000D02002000E100E0A4110020058D000815
:048508004A0F0020F6
:10850C0010B5012041020D4A1160BFF34F8FBFF32C
:10851C006F8FEA220A4B00249C520A4A0A4C54667A
:10852C000A4A11600C4908702120C000195A491CD4
:10853C00195207480749016010BDC04680E100E0B0
:10854C00600E0020AC100020E101002000E100E0F2
:0C855C00A4110020058D00086011002013
:1085680010B5002902D00020C44326E0144A116A3D
:10857800431A1449CC69A34221D9106212480068F1
:108588000A78002A07D0C0B2C409086AA04208DBEA
:108598000E4A0F480AE0FF228243D409086AA04223
:1085A800F6DAA0000B4A1018006D0B4AA300D25847
:1085B800CA610849C918486380470248046210BD67
:1085C800AC100020E40500201008005064C3000827
:0C85D80001000020A41100205CC300087A
:1085E40030B50120420222490A60BFF34F8FBFF326
:1085F4006F8FEA231F490024CC521F4B1F4D5D6629
:108604001F4B1A608C85C5431E4B1A681561546252
:108614001D4C1E4D25603D241D5D012D1FD10225DD
:108624001D55D3680343D360194B9A4206DC830774
:108634009A4209D0194B9A4206D00DE0154B9A4242
:1086440002D0154B9A4207D19468154B2340062B50
:1086540005D00404A34202D0136803431360114AF3
:1086640010702120C0000A5A521C0A5230BDC04664
:1086740080E100E0600E0020AC1000200500002026
:1086840000E100E0AC140020A4110020F18B0008EC
:10869400FF2B014000400140002C01400004004039
:0886A400070001006011002035
:1086AC0010B5002901D0022421E0124AD169431AE5
:1086BC0011494C69A3421CD9D061104800680A7852
:1086CC00534253414006C40F5C408869A04202D11A
:1086DC000B4A0C4804E0A0000B4A1018006D0B4A22
:1086EC00A300D2584A610849C918C8628047024899
:1086FC00846110BDAC100020E4050020100800506F
:10870C0064C3000801000020A41100205CC3000811
:10871C0001204102084A1160BFF34F8FBFF36F8FE6
:10872C000B4A10800548064A426606480160064816
:10873C00064901607047C04680E100E0AC100020A3
:10874C00B101002000E100E0A4110020058D00081B
:04875C004A0F0020A0
:1087600010B5012041020D4A1160BFF34F8FBFF3D6
:108770006F8FEA220A4B00249C520A4A0A4C546624
:108780000A4A11600C49087085204000195A491C9A
:10879000195207480749016010BDC04680E100E05A
:1087A000600E0020AC1000208501002000E100E0F8
:0C87B000A4110020058D000860110020BD
:1087BC0010B5002902D00020C44321E0124A91696F
:1087CC00431A1249CC68A3421CD990611048006826
:1087DC000A78534253414006C40F5C400869A042DA
:1087EC0005DAA0000D4A1018006D0D4A01E0094A87
:1087FC000948A300D258CA600849C9184862804782
:10880C000248046110BDC046AC100020E4050020F5
:10881C001008005064C3000801000020A4110020BF
:04882C005CC3000821
:1088300030B50120420222490A60BFF34F8FBFF3D7
:108840006F8FEA231F490024CC521F4B1F4D5D66DA
:108850001F4B1A608C85C5431E4B1A681561546204
:108860001D4C1E4D25603D241D5D012D1FD102258F
:108870001D55D3680343D360194B9A4206DC830726
:108880009A4209D0194B9A4206D00DE0154B9A42F4
:1088900002D0154B9A4207D19468154B2340062B02
:1088A00005D00404A34202D0136803431360114AA5
:1088B0001070852040000A5A521C0A5230BDC04632
:1088C00080E100E0600E0020AC10002005000020D8
:1088D00000E100E0AC140020A4110020F18B00089E
:1088E000FF2B014000400140002C014000040040EB
:0888F0000700010060110020E7
:1088F800B0B5002901D004242EE0194AD16A431AE0
:1089080018494C6BA34229D9D062174802680068FD
:108918000B785C425C415206D20F62405200002B39
:108928000BD0C0B2C0091418886B84420CD0A000C8
:10893800104A1018006D104A08E0FF238343D80935
:108948001418886B8442F2D1084A0948A3000B4DD9
:10895800E850D2584A63804702488463B0BDC04695
:10896800AC100020E4050020100800507CC300086B
:1089780001000020A41100206CC30008C0070020DB
:10898800012041020C4A1160BFF34F8FBFF36F8F74
:10899800124A108009480A4A42660A4801600A4891
:1089A8000821016009490A4A0A600A490A4A8A658F
:1089B800022101607047C04680E100E0AC10002051
:1089C8005501002000E100E028040050A411002017
:1089D800058D000828110020010000204A0F002002
:1089E80010B50120420210490A60BFF34F8FBFF350
:1089F8006F8FEA230D490324CC520D4B0D4C5C6656
:108A08000D4B1A600D4A08231360022313600F4AA6
:108A180010702120C0000B5A5B1C0B5208480949F2
:108A280001600948106210BD80E100E0600E00207E
:108A3800AC100020DD00002000E100E02804005018
:108A4800A4110020058D00080100002060110020FD
:108A580030B50120420210490A60BFF34F8FBFF3BF
:108A68006F8FEA230D490224CC520D4B0D4D5D66E4
:108A78000D4B1A600D4A0823136014600F4A1070DA
:108A8800852040000B5A5B1C0B52094809490160BC
:108A98000948106230BDC04680E100E0600E002049
:108AA800AC1000205D00002000E100E02804005028
:108AB800A4110020058D000801000020601100208D
:108AC80010B501214A0210480260BFF34F8FBFF36F
:108AD8006F8FEA230D480024C4520D4B0D4C5C6681
:108AE8000D4B1A60104A11702121C900435A5B1CB2
:108AF800435285214900435A5B1C43520748106280
:108B080007480849016010BD80E100E0600E0020C0
:108B1800AC1000203100002000E100E00D8C0008BE
:0C8B2800A4110020F18B00086011002057
:108B3400B0B5002906D02C4800210170C843234950
:108B44000863B0BD22498A6A821A204CE36A9A42B9
:108B54003BD988621F480168006822785342534118
:108B64004906C90F59404900002A0ED0C0B2C009B5
:108B74000D18206B85420FD01B480178012914D1B0
:108B8400A80016490818006E1BE0FF228243D00992
:108B94000D18206B8542EFD1A80011490958E162F4
:108BA4000E4909180F4808660DE0002D01D0012177
:108BB4000170A80008490958E16208490918086DBC
:108BC4000866002800D080472563B0BDE405002076
:108BD400AC100020100800506CC30008A411002041
:0C8BE4007CC30008010000205811002094
:108BF0000348044901600448102101607047C046E1
:0C8C0000A41100200100002028040050F6
:108C0C0030B584B06846C821018002AA1180518019
:108C1C003449C1807D21890041808180C831918097
:108C2C00D18031494B683148026A032B0AD88C68D1
:108C3C00022C18D0012C08D0002C20D12C4B08244D
:108C4C001C600CE000224A6019E05B0002ACE35AA5
:108C5C000C68141B9C4212D9254B08241C610A6019
:108C6C008A68521C0AE05C006D462C5B0D68551B33
:108C7C00A54204D90A6000225B1C4B608A601D4926
:108C8C004A6F006A032A0AD88B6F022B1BD0012B68
:108C9C0009D0002B05D1164A022313600DE00020E9
:108CAC00486704B030BD520002AB9A5A0B6FC31A1E
:108CBC009342F6D90E4A022313610867886F401C51
:108CCC00886704B030BD53006C46E35A0C6F041B2C
:108CDC009C42E6D908670020521C4A67886704B09A
:108CEC0030BDC046C4090000AC100020A411002007
:088CFC001804005028110020AB
:108D040070B50C48C1680C4A136A5D1A0B490A7F96
:108D14000B4C002A03D0C92D0BD3103403E01926C1
:108D24007601B54205D910252560C3600120424073
:108D34000A7770BDAC100020A41100202811002077
:048D440018040050BF
:108D48000448082101600449044A8A650221016037
:108D58007047C04628040050281100200100002058
:108D68000348044901600448102101607047C04667
:0C8D7800A411002001000020180400508D
:108D8400032000020A490A6802404A60094D0A4C5D
:108D94002868022101225204030408401340C01829
:108DA400484068600020214603F0B8FAF0E7C04666
:0C8DB4001C1002401404005032CC0008D7
:108DC00000241449204603F0ABFA1349204603F06F
:108DD000A7FA0120400411490B6802221C04134029
:108DE00004401B1953404B600B681C0413400440A3
:108DF0001B1953404B600B681C04134004401B19A3
:108E000053404B600B681C04134004401B19534033
:108E10004B60E1E7A0D00008A8D00008140400507F
:108E200080B5024801F022FF80BDC0467C130020BF
:108E300080B5024801F01AFF80BDC0463013002003
:108E400080B5024801F012FF80BDC046AC1400207E
:108E500080B5024801F00AFF80BDC04660140020C2
:108E600080B5024801F002FF80BDC0461414002006
:108E7000F0B595B003A808302C2103F065F92F4810
:108E800000682F49884201D015B0F0BD0225049535
:108E90000126039603A801F09BFC002814D00024AF
:108EA0002849204603F03CFA2749204603F038FAC7
:108EB0002649204603F034FA2549204603F030FACB
:108EC0002449204603F02CFAB0032349CA68024320
:108ED000CA60CA680240109210980868304308605F
:108EE0000868304002901496002713971297119546
:108EF000092040021090029805200407019510AD4A
:108F00002046294601F024FB1496139712960198E7
:108F10001190B00210902046294601F019FBFF2065
:108F200000060E490A688243032080071018086073
:108F3000F0060B49086015B0F0BDC0461C100020BB
:108F400000380140CCD0000842CC000881C900089C
:108F50002CC9000840CC00083410024018E400E09E
:048F600000E100E04C
:108F6400B0B5054600240A49204603F0D7F909495B
:108F7400204603F0D3F90849204603F0CFF92046F0
:108F8400294603F0CBF90549204603F0C7F9B0BDE3
:108F9400BCD0000842CC000881C9000840CC0008BD
:108FA40070B50D46064600240A49204603F0B6F97A
:108FB4002046314603F0B2F90749204603F0AEF9E2
:108FC4002046294603F0AAF90449204603F0A6F9ED
:108FD40070BDC046CCD0000881C9000840CC000850
:108FE400F0B583B0C34E00230C24C34AC34D2E6096
:108FF4007461B361F36133627362B362326070604F
:1090040001200703002904D0012974D10324640238
:1090140000E084023D46B5603461012900D8184659
:1090240002974003F06084257059002805D1802000
:1090340000213154FFF71AFF326824200190705147
:1090440010680127B843106001F016FF01283CD0D6
:10905400B06A002801D002F0FFF8B90330688268D2
:109064000A438260F90382688A4382600168A44AE1
:109074000A400260F90542680A434260B906026880
:109084000A430260FF21090642690A40263242610E
:109094000168394301608C21002474509949096A9C
:1090A4000268120709D5780500970F4602F040F9C7
:1090B4003946009F002808D130680068400720D551
:1090C400B80502F035F900281BD000248E4920464B
:1090D40003F024F98D49204603F020F98C492046F9
:1090E40003F01CF98B49204603F018F98A492046FD
:1090F40003F014F90CE01C461D46B56034618FD8AA
:109104008DE7202070518821705080203454F466FB
:109114007A4E30688021415C012915D17A49204674
:1091240003F0FCF87949204603F0F8F87849204622
:1091340003F0F4F87749204603F0F0F87649204626
:1091440003F0ECF8306810E001468031019A4A607F
:10915400026813681468BC4314607C07A34313605B
:10916400002242660A7020224A60024680329168D8
:10917400202909D18168029B994202D10169002901
:1091840002D01178012915D100245F49204603F04B
:10919400C5F86849204603F0C1F85D49204603F04C
:1091A400BDF86549204603F0B9F85B49204603F051
:1091B400B5F8FEE704465C340021C1661770036805
:1091C400564DAB4210D05B681B020DD5EFF31083F4
:1091D400019387F31088BD06066833682B43336018
:1091E400464E019B83F3108801673B026380019321
:1091F40023803546273585658568002D0BD03E07CD
:10920400B5420DD03E03B5420FD10569002D05D1FD
:109214001D46FF350CE00569002D08D1FF2507E048
:109224000569002D03D03F2502E0A18001E07F25E0
:10923400A580D16022259560EFF3108587F310880F
:109244000668B3683B43B36085F310887B07456EBB
:109254009D42019E02D1A389B34216D98368029C20
:10926400A342264D02D10369002B18D02F4C117054
:109274000467EFF3108287F31088203600680368D0
:109284003343036082F3108823E08368029CA34283
:109294001A4D02D10369002B03D0224C02E0224C68
:1092A400E5E71F4C11700467EFF3108287F3108811
:1092B40003681C6834431C6082F31088EFF3108247
:1092C40087F310883B07006884681C43846082F33A
:1092D4001088262029544720C000184A2A508D207F
:1092E4008000134A2A50A984E96129841C35A97194
:1092F40003B0F0BD1C10002000380140240C0020F5
:10930400FFFF00FCA4110020CCD0000842CC0008D0
:1093140081C900082CC9000840CC00080080004026
:1093240085B60008D5B4000817C5000889C600082A
:1093340030060020D4D0000863CE00086E1100204F
:10934400F0B587B0414F3868002808D538460C3846
:109354003F4901603F490160386800285BD401251A
:109364006E023C46143C2068B04320600220019009
:1093740003900695384800680006400E801E05904C
:1093840003A802A900F0C4FFE907002839D100911D
:10939400354632480CC8324800F002FF0326002844
:1093A40001962CD12D488268C3682D48083000F0FE
:1093B400F7FE002823D12948026943692848103060
:1093C40000F0EEFE00281AD124488269C3692448BB
:1093D400183000F0E5FE002811D12048026A436AE3
:1093E4001F48203000F0DCFE002808D11B48826AA8
:1093F400C36A1B48283000F0D3FE00280ED02E4646
:109404000099206830432060386808433860386821
:10941400019807B0F0BD012007B0F0BD0F48026B02
:10942400436B0F48303000F0BBFE00282E460099F5
:10943400E7D12068304320603868084338603868D2
:10944400410F0420884307B0F0BDC04614200240F9
:1094540023016745AB89EFCDE075FF1FC0060020EF
:0494640000F001080B
:1094680010B566490A78664802704A7842708A7868
:109478008270CA78C2700A7902714A7942718A790F
:109488008271CA79C2710A7A02724A7A42728A7AF7
:109498008272CA7AC2720A7B02734A7B42738A7BDF
:1094A8008273CA7BC2730A7C02744A7C42748A7CC7
:1094B8008274CA7CC2740A7D02754A7D42758A7DAF
:1094C8008275CA7DC2750A7E02764A7E42768A7E97
:1094D8008276CA7EC2760A7F02774A7F42778A7F7F
:1094E8008277C97FC177474A11782023C1545178C0
:1094F8002123C15491782223C154D1782323C15404
:1095080011792423C15453792524035593792624AA
:109518000355D37927240355137A28240355537AFE
:1095280029240355937A2A240355D37A2B240355E7
:10953800137B2C240355537B2D240355937B2E2416
:109548000355D37B2F240355137C30240355537CB8
:1095580031240355937C32240355D37C332403559B
:10956800137D34240355537D35240355937D3624C8
:109578000355D27D3723C2540368234AD3821B0C78
:10958800138383885383C38893830389D38343894D
:10959800138583895387438A9387838AD387C38AAA
:1095A80042241353038B44241353438B46241353ED
:1095B800838B48241353C38B4A241353C3894C24E5
:1095C8001353038A4E241353038C104C2380002B0F
:1095D80002D050230124D452036B9360828D382A21
:1095E80004D1C08D002803D0032010BD022010BD77
:1095F8006539481E8141880010BDC04600F0010849
:10960800C006002020F00108600E0020761100201E
:10961800F0B587B0314F3868002808D538460C387F
:109628002F4901602F4901603868002825D4012698
:10963800710201913D46143D286888432860022440
:1096480003940696284800680006400E401E0590C0
:1096580003A802A900F05AFE2146F407019E00283B
:1096680025D12248826A0746C36A214800F096FD40
:109678000321002805D0194F19E00121084607B039
:10968800F0BD00913A6B7B6B1948083000F086FDFD
:10969800002802D0114F009909E0BA6BFB6B1448FF
:1096A800103000F07BFD00280C4F009909D0286885
:1096B800304328603868204338603868084607B067
:1096C800F0BD28683043286038682043386038681F
:1096D800400F04218143084607B0F0BD1420024022
:1096E80023016745AB89EFCDE075FF1FC007002058
:0496F80000F801086D
:1096FC00F0B585B0804D2F68B8680224400728D497
:10970C005426A85D012824D001200390A855F868A0
:10971C00C0077A4B0BD1B868C00704D0B8681840A2
:10972C0002210143B960F86801210143F96000246A
:10973C000494B868C00742D118462F30B96801426A
:10974C000AD0A86D10210143A965E86D01242043BE
:10975C00E865204605B0F0BDB868184001210291BB
:10976C000843B86066480068000200D59CE0687E3B
:10977C00012824D06548016A3A68D2071FD10194A8
:10978C0002E03A68D2071AD1BA68D2070FD1BA6888
:10979C001A4034462E461D460B460146029802439B
:1097AC00084619462B4635462646019CBA60026A85
:1097BC00521A032AE5D33A68D207E2D1C1E7AC5575
:1097CC00A86D534901402846039D2A02029289182C
:1097DC008165C4651C233B60016D4E4A4E4E4F485B
:1097EC00C8620E634A637868102202437A602420B0
:1097FC00085C012801D102244BE00A462432157082
:10980C005078012841D102205070CC630A6810684E
:10981C000125A8431060886CCE6C4660086D0090E2
:10982C00002802D0486D8E6D46604037086C184099
:10983C0003952B4683403A4806681E430660062073
:10984C0050608B683748102B06462B4D00D03E4697
:10985C009660102B00D00746D76010680E23034388
:10986C001360496C0868C003029E02D50868304337
:10987C00086000990029214B02D008683043086029
:10988C00106803990843106005E014708020C863C9
:10989C002C461A4B184D28688168194004220A433B
:1098AC008260204605B0F0BD1648806C164902F067
:1098BC00BDFB124B401C04900498002800D156E7C5
:1098CC000498401E04900498002800D14FE7049897
:1098DC00401E04900498002800D148E70498401ECC
:1098EC0004900498002800D141E70498401E04908D
:1098FC0004980028E4D13AE714120020E8FFFF7F17
:10990C0008270140E4050020400D0300A4110020AD
:10991C00FEF0FFFFB1C5000815C50008AFC4000874
:08992C0004000240E8110020D4
:10993400F0B587B00025069554269E4FB95D0129E0
:1099440003D10224204607B0F0BD0124BC55396878
:109954008A68520714D43B694268022A18D1042247
:109964001343964A93426FD1934AD3430268D04338
:1099740018438B6A03408B620024002A68D4CCE02D
:10998400B86D20210143B965BD55204607B0F0BD2F
:10999400059204273B43884A884CA34265D1046856
:1099A40022408B6A13438B62824F22024B6993439A
:1099B40080681040824A02401A434A6122460024C9
:1099C400002A00D4A9E0012005907E4803680720FE
:1099D40080051946049001407B480292824200D0DF
:1099E40082E00598C0051A4602407DD1754A126886
:1099F400049B9A4311430143724801607548806C8B
:109A0400754902F017FB0C2141430C31069106986D
:109A1400002800D181E00698401E06900698002890
:109A24007BD00698401E06900698002875D00698AC
:109A3400401E0690069800286FD00698401E069097
:109A440006980028E7D168E002680024002A64D55B
:109A54005C4801685D4B9A4266D05D4B9A4266D081
:109A6400594B9A4259D105225FE002971F24059B66
:109A74001C400F2300930494A3404E4F3C6E01936B
:109A84009C4323460468144203934AD0E2072A46BF
:109A94005FD1A20758D4620758D4220758D4E206EB
:109AA400029A56D4A2066CD462066CD422066CD4F4
:109AB400E2056CD40294A2056BD462056BD4220532
:109AC4006BD4E2046BD4A2046BD462046BD422047E
:109AD400009A384F3DD4E20368D4A20368D46203E9
:109AE400D31712221A405FE03848029A824204D106
:109AF400059800061A46024007D03548029A824269
:109B04000BD105988005034007D12E4A1268049BA7
:109B14009A43114301432B4811E0BD55204607B039
:109B2400F0BD6200D20E14E00322920501E003228C
:109B3400D205114007229205036893435918016026
:109B4400BD55204607B0F0BD012202E0022200E02C
:109B54000322049B9A40039B1A433A66059A92088F
:109B6400FB69934200D820E7019AD2438B6A1340E1
:109B74000593A200120F049B9A40059B1A438A6224
:109B840013E70522E5E70622E3E70722E1E70822D7
:109B9400DFE7092208E00A2206E00B2204E00C2297
:109BA40002E00D2200E00E22024FD2E71022FBE772
:109BB4001122F9E714120020FFFF070004000080BF
:109BC40000FFFF0708270140001000B0004000B864
:0C9BD400002000B4E4050020400D030058
:109BE000F0B583B05422C14FB95C012902D10220E3
:109BF00003B0F0BD39688C686407BD4B00D58EE0BA
:109C0000066844689E4215D10125EE05B44266D02F
:109C10000326B605B4426BD11F24A40687682740EB
:109C2000CB680293B74C1C403C19B04FB04BA41901
:109C3000CC6061E00127FD05AC42AE4B7FD00297BE
:109C40000325AF05BC4200D089E00C46A034009447
:109C50008768AB4C01973C409E42A44F00D08CE0FB
:109C6000002C00D1B8E0019BDC0700D0BCE09C07D1
:109C700000D5C3E05C0700D5C2E01C0700D5C3E0F7
:109C8000DC0600D5C1E09C0600D5C2E05C0600D52C
:109C9000C3E01C0600D5C4E0DC0500D5C5E09C058A
:109CA00000D5C6E05C0500D5C7E01C0500D5C8E0BE
:109CB000DC0400D5C9E09C0400D5CAE05C0400D5F2
:109CC000CBE01C0400D5CCE0DC0300D5CDE09C0348
:109CD00000D5CEE05C03E41712252540CAE0CC682D
:109CE0003B46884F2740BC191F46814BCC6003E0A0
:109CF000CC68844E2640CE602C04BD6DA543BD6566
:109D000080240C604D68067B012E06D125434D60F2
:109D1000066905689D4207D0D2E0A5434D600669FB
:109D200005689D4200D0CBE0CB689B080624234009
:109D30009E40CB689B08234044699C40C1E06E4C28
:109D4000E443F5432543F40C04272740CC19A0270E
:109D5000E3592B40694D35401D43E5510BE0664BFF
:109D6000DB43F4431C43F30C04251D404B19A02591
:109D70005E5926405E515D4F83E0002C30D0019B40
:109D8000DC0733D19C07029E31D45C073AD41C0710
:109D90002E462CD4DC063AD49C063CD45C063ED439
:109DA0001C0640D4DC0542D49C0544D45C0546D452
:109DB0001C0548D4DC044AD49C044CD45C044ED426
:109DC0001C0450D4DC0352D49C0300D58AE05C030D
:109DD000E4171226264086E0019B5C00E50E4AE06F
:109DE000019B5C00E60E02E0002544E00026029D97
:109DF000B540009B5C682C435C6042E001253AE082
:109E0000022538E00226F2E735E0042533E0042697
:109E1000EDE705252FE00526E9E706252BE00626D8
:109E2000E5E7072527E00726E1E7082522E00826E1
:109E300059E009251EE0092655E00A251AE00A2600
:109E400051E00B2516E00B264DE00C2512E00C2608
:109E500049E00D250EE00D2645E00E250AE00E2610
:109E600041E00F2506E00F263DE0102502E0102618
:109E700039E011251D4F0124AC40009B1D6825438E
:109E80001D60BC6D03681B4DAB4205D101235D0411
:109E9000AC43BC651C0204E001239D04AC43BC65DB
:109EA0005C020C604D68037B012B01D1254300E06F
:109EB000A5434D600E4B066905689D4200D133E70E
:109EC00044690020B85432042243AB02DC0F9B0FDC
:109ED0001B199B00C9180B6A0B4C1C4014430C62E5
:109EE00003B0F0BD1126014F81E7C04614120020D7
:109EF0000000C07CFFFF1700FFFFC77CFFFF87004B
:0C9F0000FFFF0700FFFF3F8300F000F0B0
:109F0C00F0B582B0654A537D012B02D1022002B01C
:109F1C00F0BD02231375012757750668042E1DD159
:109F2C00019600292CD014695D4E636B002B51D522
:109F3C00336A012B46D8636B002B4BD5336A012B4C
:109F4C0040D8636B002B45D5336A012B3AD8636B31
:109F5C00002B3FD5336A022BE7D333E01469036936
:109F6C00012B76D11023194043698B401F258D405E
:109F7C003246A66BAE431E43A6631646474A6AE0BA
:109F8C001469474E3B46376A0093DD03636B2B42E3
:109F9C0035D0336ADB1B012B14D8636B2B422ED0CC
:109FAC00336ADB1B012B0DD8636B2B4227D0336A32
:109FBC00DB1B012B06D8636B2B4220D0336ADB1BD7
:109FCC00022BE3D3106A08210143116203201075A0
:109FDC0002B0F0BD0097356A336A5B1B012B0BD8BE
:109FEC00336A5B1B012B07D8336A5B1B012B03D82D
:109FFC00336A5B1B022BEFD38369636412E0356A0F
:10A00C00336A5B1B012B0BD8336A5B1B012B07D804
:10A01C00336A5B1B012B03D8336A5B1B022BEFD318
:10A02C008369236410250D40C369AB401D4EAE40BF
:10A03C00A76CB7431F43A764036AAB40FF26AE402F
:10A04C00E56CB5431D43E564009F019E0369012B3C
:10A05C0088D01023194007238B40E56B9D43836800
:10A06C003343C6681E438E402E43E663BB038B40CE
:10A07C0025689D432560406888400B4B8B402568C4
:10A08C009D4305432560C0208840216881432160A1
:10A09C0000205075177502B0F0BDC046C0070020F7
:0CA0AC00A4110020FF030000FE0F0000C4
:10A0B800F0B583B0002840D0044606462436022076
:10A0C8007070276838683049014039602F488030FF
:10A0D800A0642F4838181425294601F0A9FF8000EC
:10A0E8002A494118206401916164F8B20838294668
:10A0F80001F09EFF1F210140012528468840E064A9
:10A10800A268E168114323690B4361691943A36994
:10A118000B43E1691943236A0B43396819433960D2
:10A128000295A9038A421B4A0AD1002301990B60B0
:10A13800636010601F461D461CE0012003B0F0BD9F
:10A1480063683F211940019D29601060581E002353
:10A1580003281F461D460DD8481E810053180021AC
:10A16800D96703210140029D8D400B4805607C336F
:10A17800BC3217460020E06323656765A56530702B
:10A188000299717003B0F0BD0F80FFFF0008024014
:0CA19800F8FFFDBF8408024044090240AB
:10A1A400F0B585B059490C78002C02D0022005B0D6
:10A1B400F0BD0290039301270F707D20C100504E23
:10A1C400306A049141183C044E4D2868204216D050
:10A1D400336A03208B426CD22B6823420FD0336A3C
:10A1E4008B4266D22B68234209D0336A8B4260D2F9
:10A1F4002B68234203D0336A8B42E6D359E02868A4
:10A2040041494B1C01932B600842384651D1306AB6
:10A21400049941180120009087042868384216D018
:10A22400336A03208B4244D22B683B420FD0336AFB
:10A234008B423ED22B683B4209D0336A8B4238D2E0
:10A244002B683B4203D0336A8B42E6D331E0686823
:10A2540000990843686002990A60BFF36F8F0398FE
:10A264004860306A049941182868204216D0326A3E
:10A2740003208A4219D22A6822420FD0326A8A42C3
:10A2840013D22A68224209D0326A8A420DD22A683D
:10A29400224203D0326A8A42E6D306E02868019952
:10A2A400296019490842009808D06968009A9143C6
:10A2B40069600021154A117005B0F0BD306A049937
:10A2C40041182A6800203A42EFD0336A03228B42B5
:10A2D40013D22B683B42E8D0336A8B420DD22B68F1
:10A2E4003B42E2D0336A8B4207D22B683B42DCD03C
:10A2F400306A88421046E4D3D7E71046D5E7C04613
:10A30400A411002010200240FAC3000068110020AC
:10A31400F0B586B002468C4C2078002802D002208A
:10A3240006B0F0BD0491012323707D20C100824D4D
:10A33400286A059146181F04804C2068384216D0BC
:10A34400296A0320B1421AD2216839420FD0296AFE
:10A35400B14214D22168394209D0296AB1420ED2DD
:10A364002168394203D0296AB142E6D307E0206864
:10A3740073494E1C039626600842184604D00021F7
:10A38400714A117006B0F0BD286A0599461801207B
:10A39400029083042068184216D0296A0320B1422F
:10A3A400EDD2216819420FD0296AB142E7D221685F
:10A3B400194209D0296AB142E1D22168194203D075
:10A3C400296AB142E6D3DAE7042050601068042811
:10A3D40020D1381D616801436160286A05994218DB
:10A3E4002068384270D0296A03209142C7D221687C
:10A3F400394269D0296A9142C1D22168394263D075
:10A40400296A9142BBD2216839425DD0296A9142BE
:10A41400E6D3B4E70026F043049908609168D06855
:10A424004218914258D20096464E606830400191DD
:10A43400C9000143B81C08436060286A059946189E
:10A444002068384216D0296A0320B1426CD22168B0
:10A4540039420FD0296AB14266D22168394209D003
:10A46400296AB14260D22168394203D0296AB142D3
:10A47400E6D359E02068039921603149084252D15A
:10A48400286A059946182068184216D0296A0320BC
:10A49400B14249D2216819420FD0296AB14243D24C
:10A4A4002168194209D0296AB1423DD22168194272
:10A4B40003D0296AB142E6D336E00199491C91429E
:10A4C400204EB2D1009832E02068039921601C49E3
:10A4D400084203D0012052E7304628E0286A059953
:10A4E4004118226800201A4200D148E72E6A03224C
:10A4F4008E4216D226681E4200D140E72E6A8E4252
:10A504000FD226681E4200D139E72E6A8E4208D245
:10A5140026681E4200D132E7286A88421046E0D3FA
:10A524002DE710462BE702980499019A0A606168A6
:10A5340002229143616022E7A4110020102002400E
:0CA54400FAC3000005FEFEFF68110020B5
:10A55000F0B58CB006900B68002B00D1C7E06548C1
:10A56000069A824201D0052000E0032000900124D9
:10A5700000200246074603940B900A90019112E0D6
:10A580001343059A5C4843600B681846E0400B9DF6
:10A59000AD1C0B95121D0837641C0A9E761C0A968A
:10A5A000002800D1A3E0601E039E0990864033403E
:10A5B0000793E9D00B9B08974D6803212F460F4066
:10A5C000781E01280592029519D804941C469940DA
:10A5D000069A90688843019BDB68A340034393601D
:10A5E000E806049CC00F099B98405368B343164685
:10A5F000059A03437360CB430A9845000BE0084675
:10A600001D469840C343032F069E04D104930B9D1F
:10A610000F4601991CE0F0680493184001998B687B
:10A62000AB400343F360022F12D11C2010400F27D0
:10A630008740099BDB089B00F3181E6ABE430F6925
:10A6400087403743069E1F624B6803271F4000E088
:10A65000029BAF403068049D284038433060980327
:10A66000800F089F90D0182038400F268640032383
:10A67000099F9F43204AD7193B6EB3436037052695
:10A680003607069AB2420AD01D4EB24205D01D4E80
:10A69000B242009E04D1022602E0012600E000261C
:10A6A00086401E433E60154806684868C30302D5CD
:10A6B000079A164301E0079A9643089F0F4B1E60C6
:10A6C0005E68830301D5164300E096430B4B5E6042
:10A6D000094B1E68C30201D5164300E09643064BA2
:10A6E0001E605B68800200D54AE7934349E70CB0DF
:10A6F000F0BDC046000C0050001802408018024017
:08A700000004005000080050A5
:10A70800F0B588B001210022164617460291009044
:10A7180024E0069DB5402B4C2068284320601C206F
:10A728003840059A82400398C00880002018036AC0
:10A7380093430362A068A843A0606068079B98439E
:10A748006060E068A843E0600098049A0346CB4044
:10A758000832B61C3F1D491C002B2DD04D1E029BF4
:10A76800AB401C460440F1D00793182004921040D7
:10A778000F22059282400323039506939D430F4BB6
:10A788005B1901931D6E1540012383409D42C0D182
:10A79800019D60350A4B1868A04318605868A043AB
:10A7A8005860064B1868A04318605868A043586062
:10A7B800286890432860ACE708B0F0BD0018024054
:08A7C80080180240000400505B
:10A7D000F0B586B00746036899038D4A03D400207C
:10A7E000D90761D166E00497012528071446183C73
:10A7F00021680140039106D121680143216021684D
:10A800000140059105990194029000952E02814C1A
:10A81000216831432160804F3D6A216831421AD15D
:10A82000396A491B0320022933D82168314212D1E9
:10A83000396A491B02292CD8216831420BD1396A67
:10A84000491B022925D82168314204D1396A491BA4
:10A850000229E2D91DE00320010294680C4004990A
:10A860000E6B10D0B4420BD094680099090495681F
:10A870000D43956095688D43956068490C409460E0
:10A88000E10700D09DE09068644908403043906043
:10A8900000200399002904D1019D2968029CA1434D
:10A8A0002960049FD90705D011680324A1437C685F
:10A8B0000C43146099070BD4D90611D4990518D408
:10A8C00059051FD4990626D4012459042DD43BE000
:10A8D00011680C24A143BC680C431460D906EDD563
:10A8E0000321890214688C43F9682143116099059A
:10A8F000E6D50321890414688C43B96921431160AA
:10A900005905DFD50321090514688C43F9692143F2
:10A9100011609906D8D50321090314688C4339695D
:10A9200021431160012459040ED511683D4D294081
:10A930003E6A31431160691C8E4205D121041546DF
:10A94000483D2E680E432E60190305D51168402539
:10A95000A9437D6A0D431560A50599020FD51168BD
:10A96000A943BE6A31431160AE4208D1210603916A
:10A970001646483E049737680F433760049F2B42C2
:10A980000CD025061168A943FE6A31431160AE421E
:10A9900004D1114648390E682E430E6019050ED5B4
:10A9A000A10303239B0315689D437B691D43156029
:10A9B0008B4204D12104483A13680B43136006B05C
:10A9C000F0BD3C6A164D9168890700D55BE7396A8E
:10A9D000091BA94200D95CE79168890700D552E7B5
:10A9E000396A091BA94200D953E79168890700D544
:10A9F00049E7396A091BA94200D94AE791688907E2
:10AA000000D540E7396A091BA942DCD941E7C046B5
:10AA10005410024000700040A4110020FFFCFFFF12
:08AA200088130000FFFFFF3F57
:10AA2800F0B581B0002823D001463C314A78002A8D
:10AA380021D002224A7003681E6801229507AB42A2
:10AA480005D0824CA34202D0814CA34241D170244C
:10AA5800A643846834437F4EB3423EDD7E4DAB420D
:10AA680030DC7A4DAB4240D07C4DAB423DD08CE0DF
:10AA7800012001B0F0BD0A7003686B4A934263DCA1
:10AA880001229407A34200D181E06B4CA34200D17C
:10AA980086E06A4CA342CCD1694B1C6820252C4324
:10AAA8001C601B682B400093009BFF231B04654C14
:10AAB80025689D4303239B05EB1823609204624B92
:10AAC8001A60B6E75B4DAB420FD0594DAB420CD084
:10AAD8005BE034465F4EB342C0DCAB4205D05C4D10
:10AAE800AB4202D0514DAB424FD103252D02AC43AE
:10AAF8000669264305463E35044644348027BE434E
:10AB0800876937431F60C668DE6246689E62544E96
:10AB18009E190A27FE41072E06D81746B740E12698
:10AB2800374201D0406918635A6122712A706A70ED
:10AB3800AA70EA702A716A7122706270A270E2705B
:10AB48004A70002001B0F0BD384A93423ED0384ADE
:10AB5800934252D0374A934200D06AE701229304C5
:10AB6800374C65681D43656064681C400094009B11
:10AB7800FF231B04334C65689D4303239B05EB1897
:10AB880063609205304B1A6053E72646B2E72C4BB8
:10AB98001C6814431C601B6813400093009A48E724
:10ABA800274B1C6810252C431C601B682B40009306
:10ABB800009BFF231B02234C25689D4303239B0313
:10ABC800EB1823605204204B1A6032E70122D303AA
:10ABD8001B4C65681D43656064681C400094009BBD
:10ABE800FF231B06174C25689D4303239B07EB187F
:10ABF8002360D204144B1A601BE701225304104C43
:10AC080065681D43656064681C400094009BFF23D1
:10AC18001B020C4C65689D4303239B03EB18636080
:10AC28005205094B1A6004E7FF1F0040002000404E
:10AC3800004401400048014000100040001400405A
:10AC48003C10024010E400E000E100E0002C01406C
:10AC580000040040FF2B0140FF4301400040014039
:04AC680000D4FEBF57
:10AC6C00F0B583B004460120C54321680A699207F8
:10AC7C0007D5CA68920704D56A1E0A61002222779A
:10AC8C008A690A69520707D5CA68520704D5EA1EB1
:10AC9C000A61002222778A690A69120707D5CA68F5
:10ACAC00120704D5EA1F0A6100222277CA690A69D1
:10ACBC00D20608D5CA68D20605D52A460F3A0A61CB
:10ACCC0000222277CA690A69D20771D0CA68D207F2
:10ACDC006ED00D61CA688243CA600A6A504E324215
:10ACEC0006D10A6A4F4B1A4202D10A6882430A60A3
:10ACFC003D23E0544C4A914243D04C4A1268914255
:10AD0C004AD04B4A1268914251D04A4FB9424CD06A
:10AD1C00494FB9424BD1EA21019100210291474997
:10AD2C00019F0092029ACA53009A4449029F8F8550
:10AD3C00D7688743D760434F41494F664249434FD9
:10AD4C000F60176A374206D1166A364F3E4202D15F
:10AD5C00166886431660364EF0541561029951629E
:10AD6C00F15C012923D10221314EF154D168014308
:10AD7C00D16037498A4240DC81078A4243D0374947
:10AD8C003FE0EA212D4A50522D49364B4B669085B7
:10AD9C002D48354901600AE02848022181852A485E
:10ADAC00426800200121904701E030490870216879
:10ADBC000869000605D5C868000602D528467F3804
:10ADCC0008610869C00505D5C868000602D5284683
:10ADDC00FF3808610869400605D5C868400602D5E9
:10ADEC0028463F3808610869800604D5C868800683
:10ADFC0001D51F3D0D6103B0F0BD16498A4202D04A
:10AE0C0015498A4207D19368154919400629CED0B5
:10AE1C0003049942CBD0116801431160C7E7C046C7
:10AE2C0011110000440400000010004030130020F9
:10AE3C00AC1400200048014000440140600E00208A
:10AE4C00AC10002005000020A4110020F18B00089C
:10AE5C00FF2B014000400140002C01400004004049
:10AE6C00070001003D020020698D000864110020DC
:10AE7C00F0B583B0E24D2E683068E24A0240A86813
:10AE8C002969014368690843E96908431043306044
:10AE9C0003200190000372688243E86810437060DD
:10AEAC00D94A00239642184600D0286AAC6904435C
:10AEBC00B068D64F07402743B760F06A0F24A04311
:10AECC006F6A3843F062D248864212DDD14886421E
:10AEDC0016D096425CD0D048864210D1D148C06C76
:10AEEC008007000FD04B1B58D04C964202970BD1C9
:10AEFC005CE0CA4886424FD0C948864200D0102335
:10AF0C00CA4C9642029751D00127F80381421FD1B7
:10AF1C00082B00D965E15B007B449B885B009F4458
:10AF2C00080060012F016001740060016001600184
:10AF3C008100C048846CBB480068800A1C21014019
:10AF4C00BD4840581F210140CC4000D018E147E1DA
:10AF5C00082B00D945E15B007B449B885B009F4438
:10AF6C00080040012F0140016300400140014001F5
:10AF7C007000B048846CAB480068800A1C2101400A
:10AF8C00AD4840581F210140CC4000D018E127E1CA
:10AF9C00A448C06C000A01E0A248C06C0C2303401A
:10AFAC00A148C358A14C96420297ADD10127082B5A
:10AFBC0000D916E15B00C0467B449B885B009F4434
:10AFCC0008001001B600100117001001100110014B
:10AFDC00B4009848846C93480068800A1C21014096
:10AFEC00954840581F210140CC4000D09FE0F7E02D
:10AFFC008C4B18688006400F25D01968382001400A
:10B00C0008298B4A25D1144691E0864B196889068C
:10B01C00490F3CD01A6838210A40082A844A42D188
:10B02C001446ADE00446ABE07E4B19688906490F27
:10B03C0033D01A6838210A40082A7D4A52D1144666
:10B04C00BEE00446BCE0083B18688004400FC440D6
:10B05C006DE019680140102963D1586801990840C6
:10B06C00032800D0224658684006400F411C104669
:10B07C001C4600F0DBFF61684904490E48436168D7
:10B08C00490F491C00F0D2FF040050D1A8E0083B46
:10B09C0018688004400FC44072E0083B18688004B4
:10B0AC00400FC4408CE01B680B40102B5CD15D4BF7
:10B0BC00586801990840032800D022465868400679
:10B0CC00400F411C10461C4600F0B0FF616849045B
:10B0DC00490E48436168490F491C00F0A7FF040062
:10B0EC004ED17DE01B680B40102B5DD14D4B586849
:10B0FC0001990840032800D0224658684006400FAA
:10B10C00411C10461C4600F091FF61684904490E31
:10B11C0048436168490F491C00F088FF04004FD177
:10B12C005EE019680140202963D10120C403029814
:10B13C0040004249095A204600F078FF6A6801999C
:10B14C00514388424DD3110388424AD8010E54080A
:10B15C00000200230019594100F08CFF39494118B5
:10B16C00394A91423BD33CE02E4B1A680A40202AC4
:10B17C00044605D018680840182831D17D200402F7
:10B18C00029840002D49095A204600F04FFF40001C
:10B19C0069684A08101800F049FF2949014020D07D
:10B1AC000007400F08431AE01E4B1A680A40202A79
:10B1BC00044605D018680840182811D17D200402D7
:10B1CC00029840001D49095A204600F02FFF69687B
:10B1DC004A08101800F02AFF80B2102801D3F06042
:10B1EC0000270020286768671848A866384603B00F
:10B1FC00F0BD196801401829F2D17D20040296E7B0
:10B20C001C100020F369FFCF00800040FFF4FF11F9
:10B21C00FF4B0040004C004000380140004400400F
:10B22C00004800400810024010C400080024F4003C
:10B23C0000127A00E4050020F0C3000824C70008BF
:10B24C00F0FF000000FDFFFF00FD0F0001000100FA
:10B25C0030B53448816ACA070CD18A0714D44A071E
:10B26C001CD40A0724D4CA062CD48A0634D44A0621
:10B27C003CD44CE00122520403685C689443C26ADB
:10B28C0022435A608A07EAD50122120403685C68DB
:10B29C009443026B22435A604A07E2D5012292047E
:10B2AC0003685C689443426B22435A600A07DAD500
:10B2BC000122D20303685C689443826B22435A6078
:10B2CC00CA06D2D50122120303689C689443C26B50
:10B2DC0022439A608A06CAD50122520303689C68ED
:10B2EC009443026C22439A604A0610D5012213053E
:10B2FC00026854689C43456C2C4354609D4206D1B3
:10B30C0003235B0554689C43836C234353600906F9
:10B31C0007D50121C904026853688B43C06C1843DC
:08B32C00506030BD1C10002030
:10B33400F0B502462E480568EC691440002094429A
:10B3440000D1F0BD0124E6022A4F03E0EB6913406B
:10B354009342F6D03B6A5B1A5B0E25D12B685B07E0
:10B36400F4D5EB693342F1D02E62EFF3108084F30D
:10B3740010880D2149011E4D2A6813688B43136000
:10B3840080F31088EFF3108084F3108829688A68AA
:10B39400A2438A6080F31088842020212950284603
:10B3A4008C30294688311AE0EFF3108084F310883A
:10B3B4000D2149010E4D2A6813688B43136080F3F5
:10B3C4001088EFF3108084F3108829688A68A243F8
:10B3D4008A6080F310882846883029468431802288
:10B3E4000023AB5420220A6002600320F0BDC04653
:08B3F4001C100020A411002030
:10B3FC0070B58421415821291AD1014656318A8AC7
:10B40C00002A15D0174B02E0521E140410D00C88E1
:10B41C00002C0ED00468E5692D06F5D5056D2E8837
:10B42C001E40A662AC1C04650C88641E0C80EBE705
:10B43C0070BDEFF31081012282F31088D3050468EC
:10B44C00A5689D43A56081F31088EFF3108182F30A
:10B45C0010880068026840231343036081F310884E
:08B46C0070BDC046FF010000A5
:10B4740030B58421415821290FD1014656310A881B
:10B48400002A0BD0026D1388104C1C4003689C6288
:10B49400921C02650888401E088030BDEFF31081BD
:10B4A400012282F3108803681C688025AC431C6069
:10B4B40081F31088EFF3108182F31088006802682A
:10B4C40040231343036081F3108830BDFF01000063
:10B4D400F0B587B00268D169146895688823C358A9
:10B4E400222B00D09FE0059507465E37202200926C
:10B4F4007A89002A00D19CE0009A114000D198E09A
:10B5040005468835798804910122059911400591F1
:10B51400069211020C400397019402E0890600D4BC
:10B5240087E00168496A049A1140826D1170398874
:10B53400491E3980816D491C81650668F1694A0795
:10B5440036D067426741CB07069B00D03B46002BB1
:10B5540004D1012333626F681F436F60059B5F4210
:10B564005F418B07069B00D53B46002B05D1022388
:10B5740033626B6804271F436F60059B5F425F4122
:10B58400002A069A0CD53A000CD1042232626A6869
:10B59400022313436B606A68002A039F06D107E005
:10B5A400002AF2D06A68002A039F01D000226A6050
:10B5B4003A88002AB2D1EFF31083012282F3108873
:10B5C400160207683C68B4433C60039F83F3108809
:10B5D400EFF31083029382F310880468A6682B4665
:10B5E400254D2E401D46A660019C029B83F31088C6
:10B5F400009B2B6000260667C36E012B8ED1C666A6
:10B60400EFF3108382F310880468266810229643AF
:10B614002660019C83F310880668F369DB0600D476
:10B624007CE732627AE7906908210143916107B0AF
:10B63400F0BD39880029FAD07A899142F7D2EFF324
:10B644001081012282F310880B4B5B1C0468A568EF
:10B654001D40A56081F3108808490167EFF310814C
:10B6640082F3108800680268009B1A43026081F329
:10B67400108807B0F0BDC046FEFFFFEF89C6000882
:10B68400F0B587B00268D169146895688823C358F7
:10B69400222B00D09FE0059507465E3720220092BA
:10B6A4007A89002A00D19CE0009A114000D198E0E8
:10B6B4000546883579880491012205991140059140
:10B6C400069211020C400397019402E0890600D40B
:10B6D40087E00668716A049A1140826D1180398886
:10B6E400491E3980911C8165F1694A0736D0674249
:10B6F4006741CB07069B00D03B46002B04D10123B6
:10B7040033626F681F436F60059B5F425F418B0725
:10B71400069B00D53B46002B05D1022333626B68A0
:10B7240004271F436F60059B5F425F41002A069A0E
:10B734000CD53A000CD1042232626A680223134306
:10B744006B606A68002A039F06D107E0002AF2D0E2
:10B754006A68002A039F01D000226A603A88002A9E
:10B76400B4D1EFF31083012282F310881602076824
:10B774003C68B4433C60039F83F31088EFF3108369
:10B78400029382F310880468A66803462846264D6F
:10B794002E4005461846A660019C029B83F3108840
:10B7A400009B2B6000260667C36E012B8ED1C666F4
:10B7B400EFF3108382F310880468266810229643FE
:10B7C4002660019C83F310880668F369DB0600D4C5
:10B7D4007CE732627AE7906908210143916107B0FE
:10B7E400F0BD39880029FAD07A899142F7D2EFF373
:10B7F4001081012282F310880B4B5B1C0468A5683E
:10B804001D40A56081F3108808490167EFF310819A
:10B8140082F3108800680268009B1A43026081F377
:10B82400108807B0F0BDC046FEFFFFEF17C5000843
:10B83400F0B589B015460746012607919142049652
:10B844001DD31C4602260846294600F0F3FBA842F5
:10B8540014D3294600F0EEFBA8420CD3294600F08D
:10B86400E9FBA84209D3294600F0E4FB361DA842AF
:10B87400EAD2761E02E0761C00E0B61C23460F983E
:10B884000E9C03939E4200D81E4604990140002C4E
:10B894000595049137D0002935D12021800704D49F
:10B8A4000D46039800280AD003E0302503980028A9
:10B8B40005D00D4603E0641EF868002823D4002C4C
:10B8C40021D0A6421FD27A68B968481C904203D995
:10B8D40008469042EFD108E03A685554B860F968D8
:10B8E400491CF9607A689042E5D13968386900F0FA
:10B8F400FBFCB968884202D10020B860DBE7002075
:10B90400C043F860641EF8680890002800D5AFE0D2
:10B91400069702960127059D079E0194039C012C1E
:10B924000DD96F43601E012811D96F43A01E012851
:10B9340026D96F43E01E012824D9241F1CE0304679
:10B94400394600F077FBA8421ED36F4300E004465B
:10B954003046394600F06EFBA84215D36F4330469B
:10B96400394600F067FBA8420ED36F433046394690
:10B9740000F060FBA84207D36F43012CDFD9D0E766
:10B984000446ECE70446F1E70698856807963046D6
:10B99400394600F04FFB0446069B58686A1C8242F5
:10B9A40008D92A46089982420FD0154608910029E1
:10B9B40019D528E03248005D196848559A60D8685E
:10B9C400411CD96058688242EFD1069E31683069C3
:10B9D40000F08AFCB568A84211D10025B560F16871
:10B9E400089100290FD47C43079E361B3846059CDA
:10B9F400214600F01FFBA7420746C7D203E0002000
:10BA0400C0430890F06004980028029F069C0198A7
:10BA14002ED0002806D12BE015460898089000285F
:10BA2400304625D4461E864222D2874220D2606800
:10BA34006A1C824203D92A468242EDD10AE0206878
:10BA440020214155A260E068401C0890E0606068D5
:10BA54008242E1D12168206900F046FCA168884255
:10BA640008D10025A560E068089000283046D9D5A3
:10BA740009B0F0BD0020C043E06009B0F0BDC0468D
:04BA8400E8D00008FE
:10BA880082B0F0B5FFB0FFB091B0FFAC2C340D46DA
:10BA9800684868440260684868440360FFA85430F6
:10BAA800099000226548684402606548684402605D
:10BAB800644819306449694408600AA82060E26053
:10BAC800079407E02346FFF7B1FE079CE268002AC7
:10BAD80000D57FE229786D1C25290CD00029079C08
:10BAE80000D16EE26268A368581C90422DD91846AE
:10BAF8009042EAD132E00692002729780A46233A92
:10BB08000D2A15D80220C0467A441279520097446B
:10BB18000B0F0F0F0F0F0F0F0D0F090F0F06074316
:10BB28006D1CEAE70120FAE70820F8E70420F6E7A9
:10BB38000920C0430A463A3A0024824219D22646CE
:10BB48002A462E292CD0154631E02268D154A0600F
:10BB5800E168491CE16062689042B6D121682069B9
:10BB680000F0C0FBA168884200D033E20020A0604A
:10BB7800ABE700260A2256437618303E69780B4612
:10BB88003A3B834200D28DE072435618303EAA1CDD
:10BB9800A9780B463A3B83421546EBD22E29D2D1DF
:10BBA800537819463A39814200D386E0551C2878E3
:10BBB800FB2102460A40682A60D1687802460A409A
:10BBC800682A00D073E0A87802460A40682A00D0A4
:10BBD800A7E0E87801402D1D6829E8D001465839CA
:10BBE800202950D84900C0467944898849008F44A3
:10BBF8002E002D002D002D002D002D002D002D00D4
:10BC08002D002D002D0038009E002D002D002D0048
:10BC18002D002D002D002D002D002D002D002D00B4
:10BC2800C2002D002D00CE002D00FB002D002D00A0
:10BC38002E00C046500400005404000038040000E0
:10BC480030040000E70300002C0400003DE70998D9
:10BC5800011D0991016800960197FFA82C30102258
:10BC680030E7099B181D0990079C6268A168481C69
:10BC7800904212D81A6823685A5468E76D1C014626
:10BC880058392029AED9252800D01EE7079C6268BC
:10BC9800A168481C904200D8B4E00846904200D001
:10BCA80013E75BE76A1C2E2900D179E74BE7AD1C47
:10BCB800014658392029E6D894E7511D08910024F7
:10BCC8000A225443E418303C0899CD1E01462878CE
:10BCD80003463A3B8B4200D269E754432418303C70
:10BCE8000898851E2B7818463A38884200D25EE7B5
:10BCF8005443E418303C0898451E2B7818463A38C7
:10BD0800884200D253E76243D418303C0898021D99
:10BD1800037818463A38884208460892D0D2151F48
:10BD280045E7ED1C014658392029ACD85AE709984F
:10BD3800011D09910168C817049141400A1A0A2A8D
:10BD48005CD30423642AA84960D3A648824200D859
:10BD5800CBE08A425BD310460893059200F068F95D
:10BD6800089B1B1DA149059A8A420246EAD8DB1E98
:10BD7800A3424ED94EE00998011D0991016800209F
:10BD8800082300930190FFA82C3010229BE6099805
:10BD9800011D09910468079E069F0EE0316830690D
:10BDA80000F0A0FAB168884200D013E10020B0602A
:10BDB800F768641C002F00D587E62178002900D198
:10BDC80083E67268B368581C904203D918469042BB
:10BDD800EFD1E3E73268D154B060F1684F1CF760E7
:10BDE80072689042E5D1D9E70998011D0991016867
:10BDF80000960197FFA82C300A2263E60123A3428C
:10BE080007D907E0226825235354A0E69B1EA342C6
:10BE180000D82346002E04D00498002803D400201C
:10BE280002E0002105E0012004213940890801438E
:10BE3800711A022038400390079E089301D0002C05
:10BE480003D0F80701D1002926D10498002854D43A
:10BE5800780779D505917268B168481C904237D93E
:10BE68000846904260D006980599069000286BD540
:10BE78002BE6079E3168306900F034FAB1688842D1
:10BE880000D0A7E00020B060F0680690069800286F
:10BE98000599089B00D518E6481E884229D28B428E
:10BEA80027D20590079E7268B168481C904203D952
:10BEB80008469042EAD1DCE7326820235354B06048
:10BEC800F168491C0691F16072689042DED1D0E7B2
:10BED80032682B235354089BB060F168491C0691C3
:10BEE800F160726890421FD0BDE75B1EA34290D9F3
:10BEF80090E7079E04980028AAD505917268B16852
:10BF0800481C904201D9084609E032682D23535451
:10BF1800089BB060F168491C0691F1607268049949
:10BF28004942049190429ED13168306900F0DAF9B3
:10BF3800B16888424ED10020B060F068089B05992E
:10BF48000690002800D5C0E50398002805D00120F8
:10BF58003840204301D1002917D100910197FFA84B
:10BF68002C300A220499ADE53168306900F0BAF93D
:10BF7800B16888422ED10020B060F0680690089B16
:10BF880006980028059900D59FE5481E8842E4D206
:10BF98008B42E2D205907268B168481C904203D97E
:10BFA80008469042ECD1DFE7326830235354089BAF
:10BFB800B060F168491C0691F16072689042DFD167
:10BFC800D2E7002A06D0A268002A03D000200AA9D6
:10BFD80000F088F97FB07FB011B0F0BC01BC02B0AE
:10BFE8000047C046E7030000102700009F860100B5
:10BFF800CA1751408B1A17D0C1174A409446484077
:10C00800411A48081A0000E052008242FCD9002078
:10C0180000E05208914200D3891A40419A42F8D16F
:10C0280062465040801A704710B500F075F810BD90
:10C038000A0015D00300400800E052008242FCD9F3
:10C04800002000E052089B1A06D340418A42F9D1E9
:10C05800704752089B18F8D200188A42F9D17047E5
:08C0680010B500F059F810BDFD
:10C0700038B504004D42FFF7DFFF4543611938BD75
:10C08000002B09D1002907D110B51100FFF7F0FFEF
:10C090000A000021002310BD70B400240125ED0723
:10C0A000002B07D1002905D0834203D213000022C0
:10C0B0002C0000250026A419994200D1904212D9E3
:10C0C00092185B4103D2EE076D086408F3E7DE07C0
:10C0D0005B08520892190126F6079B1903E0DE0758
:10C0E0005B0852089219801A994103D364416D414B
:10C0F000F5D30FE024196D410AD2DE075B08520820
:10C10000921980185941F5D364416D41E7D301E09C
:10C110008018594102000B002000290070BC7047B4
:08C12000002000217047C04619
:10C12800411C02780130002AFBD1401A7047C046F2
:10C13800002A03D0013A8B5C8354FBD17047C04678
:10C1480000220B0011001A00002A02D0013A815483
:04C15800FCD170475F
:10C15C0003231048104A03614361104B8261C36191
:10C16C008023DB000362002383624362C3620266A6
:10C17C000B4A53214266102282660367094AC36642
:10C18C00436700E0D17BC1540133013A102BF9D144
:10C19C007047C046740F002034C4000824080020E7
:08C1AC00F814002050C4000843
:10C1B400F8B54746CE46C56883680400406899468A
:10C1C4005B1B80B50E00170098464019934207D9AF
:10C1D400FFF7B0FFED19E560C0BCB946B046F8BD45
:10C1E4001A00FFF7A7FF4B463100ED19ED1A2A009C
:0CC1F40060684144FFF79EFFEDE7C04685
:10C20000F8B54746CE46002380B58846070016009D
:10C210009946C56884681BE0013B5B1B641BB44204
:10C2200000D934009C4200D91C00786822004146A5
:10C230004019FFF781FF2D19A144A044361BBC68AB
:10C24000631B5A1E93415B421D40FD60002E06D0C9
:10C250003B699D42E0D3013B1B195B1BDEE748466F
:08C26000C0BCB946B046F8BDB0
:10C2680070B50600431C5C00E418E00074001C4B29
:10C27800A419E400C0181B19DC6A1500012C06D0AB
:10C28800022C1FD0002C10D00024200070BD9A6A08
:10C298005C6AA2421FD9013A121B2C00954200D9B0
:10C2A80014002200FFF782FFEFE79A6A5E6AB24243
:10C2B8000CD9013A961BB542E7D82A00FFF776FF5A
:10C2C8002C00E2E7FFF798FF0400DEE71B6AD218AC
:10C2D800013A961BEFE71B6AD218013A121BDCE7FA
:04C2E800740F0020AF
:10C2EC00F8B50B4B04001B780D001600002B0CD07E
:10C2FC00EFF31087012181F3108832002900200010
:10C30C00FFF7ACFF87F31088F8BDFFF721FFEFE7CD
:04C31C00740F00207A
:10C32000F8B5050008000C00FFF7FEFE0A4B0600FA
:10C330001B78002B0CD0EFF31087012181F31088BC
:10C34000320021002800FFF78FFF87F31088F8BD27
:0CC35000FFF704FFEFE7C046740F002069
:08C35C000A000000B80B00000C
:08C3640001000000640000006C
:10C36C000A000000B80B0000B80B0000B80B00006E
:10C37C000100000064000000640000006400000084
:10C38C00004B0000650001000100E8030000000004
:10C39C0000009600CC00DC0568024803A4062002CD
:04C3AC00000000008D
:10C3B000000000000000000000000000000000007D
:10C3C000000000000000000000000000000000006D
:10C3D0000100000002000000030000000400000053
:10C3E000060000000700000008000000090000002F
:10C3F000000000000000000000000000000000003D
:10C400000100000002000000030000000400000022
:10C41000000000000400000002000000080000000E
:10C42000034C206804348047FBE7F6F799FEFEE7EB
:04C43000F8D0000838
:09C434005465726D696E616C00C3
:10C43D004465766963652049443A20756E6B6E6F6D
:03C44D00776E0007
:10C450000000000000005454522052454747455305
:01C4600000DB
:10C46100547279696E6720746F207265737461729A
:03C47100742E0026
:06C47400F6F724FED2E7FA
:02C47A00FEE7DB
:02C47C00FEE7D9
:02C47E00FEE7D7
:02C48000FEE7D5
:02C48200FEE7D3
:02C48400FEE7D1
:02C48600FEE7CF
:02C48800FEE7CD
:02C48A00FEE7CB
:02C48C00FEE7C9
:02C48E00FEE7C7
:02C49000FEE7C5
:02C49200FEE7C3
:02C49400FEE7C1
:02C49600FEE7BF
:02C49800FEE7BD
:02C49A00FEE7BB
:02C49C00FEE7B9
:02C49E00FEE7B7
:02C4A000FEE7B5
:02C4A200FEE7B3
:02C4A400FEE7B1
:02C4A600FEE7AF
:02C4A800FEE7AD
:02C4AA007047D9
:02C4AC007047D7
:10C4AE0010B5816A8B6D8A6D5024234205D0D20659
:10C4BE0012D4096D496B884710BD012043021A43FF
:10C4CE008A650A68D3681B059B0F05D18B7E002BEE
:10C4DE0002D113681B0700D410BD93685B0709D403
:10C4EE00583153680C24A3435360FF2302330A6868
:10C4FE009A4305E08A6D202313438B65CA6D5C3128
:06C50E0002430A6010BDAB
:02C5140070476E
:10C5160070B588214158222901680FD102465E3242
:10C526005388496A1940836D19801188491E118004
:10C53600991C81651188002905D070BD886908227B
:10C5460002438A6170BD02468832EFF310830121EF
:10C5560081F310880924640105682E68A6432E60BD
:10C5660083F31088EFF3108381F310880468A568BD
:10C576008D43A56083F31088202313600022026791
:10C58600C36E012BD9D1C266EFF3108281F31088F6
:10C5960003681C6810218C431C6082F310880068B5
:0AC5A600C269D206C9D5016270BD5A
:10C5B000806A816D40220A438265C16D04220A436C
:04C5C000C265704799
:10C5C40030B584214158212904D1014656318A8A43
:10C5D400002A03D130BD521E1304FBD00B88002B5C
:10C5E4000CD00368DC692406F5D5046D25789D62BA
:10C5F400631C03650B885B1E0B80ECE7EFF3108173
:10C60400012282F31088D3050468A5689D43A560C0
:10C6140081F31088EFF3108182F3108800680268B8
:0CC6240040231343036081F3108830BDF5
:10C6300030B58421415821290DD1014656310A884F
:10C64000002A09D00268036D1C7894625A1C0265A6
:10C650000888401E088030BDEFF31081012282F36C
:10C66000108803681C688025AC431C6081F3108827
:10C67000EFF3108182F310880068026840231343AF
:08C68000036081F3108830BD56
:10C6880070B5882141582229016810D102465E32CE
:10C698005388496A1940836D19701188491E1180A1
:10C6A800816D491C81651188002905D070BD886994
:10C6B800082202438A6170BD02468832EFF3108374
:10C6C800012181F310880924640105682E68A643B6
:10C6D8002E6083F31088EFF3108381F310880468C9
:10C6E800A5688D43A56083F310882023136000227A
:10C6F8000267C36E012BD9D1C266EFF3108281F3B2
:10C70800108803681C6810218C431C6082F3108811
:0CC718000068C269D206C9D5016270BD7C
:10C72400010002000400060008000A000C001000CA
:08C7340020004000800000011C
:10C73C004144432063616C6962726174696F6E205D
:07C74C006572726F7221009B
:10C753005374617274696E6720566563746F7220D7
:10C763005461626C6520636F7079696E67206672CD
:10C773006F6D20464C41534820746F2052414D2E1B
:03C783002E2E0057
:10C786004D6F646520302069732073656C65637432
:10C7960065642E204175746F2D7265636F6E6E65CC
:0BC7A6006374206973204F46462E008C
:10C7B1004D6F646520312069732073656C65637406
:10C7C10065642E204175746F2D7265636F6E6E65A1
:0BC7D1006374206973204F46462E0061
:10C7DC004D6F646520322069732073656C656374DA
:10C7EC0065642E204175746F2D7265636F6E6E6576
:0BC7FC006374206973204F46462E0036
:10C807004D6F646520332069732073656C656374AD
:10C8170065642E204175746F2D7265636F6E6E654A
:0BC827006374206973204F46462E000A
:10C832004D6F646520342069732073656C65637481
:10C8420065642E204175746F2D7265636F6E6E651F
:0BC852006374206973204F46462E00DF
:10C85D004D6F646520352069732073656C65637455
:10C86D0065642E204175746F2D7265636F6E6E65F4
:0BC87D006374206973204F46462E00B4
:10C88800555020627574746F6E206973206C6F6EDA
:0BC89800672D707265737365642E00DD
:0BC8A30056613A20253664206D5600D7
:0BC8AE0056623A20253664206D5600CB
:0BC8B9004441435F413A2025346400F5
:0BC8C4004441435F423A2025346400E9
:03C8CF004F5000C7
:03C8D200434C00D4
:03C8D500424100DD
:03C8D800414200DA
:03C8DB00257300C2
:03C8DE004F5400B4
:03C8E1004F4300C2
:03C8E4004F4C00B6
:03C8E7004C4200C0
:10C8EA0043757272656E742063616C6C6962726101
:10C8FA0074696F6E2073657175656E6365207374F4
:07C90A0061727465642E00E8
:10C91100095B2534645D2053616D706C656420761C
:0BC92100616C75653A202534640A0043
:0BC92C0048414C206572726F722100C0
:10C9370053415645204C4F434B2D4B455920434FB0
:07C947004D4D414E442E004E
:10C94E0043616E6E6F7420726573746F72652064CE
:10C95E00656661756C742073657474696E67732097
:10C96E0066726F6D20464C415348206D656D6F7237
:03C97E007921001C
:03C981003A200059
:10C984004465766963652049443A2053544D3332F3
:10C9940047304231206F722053544D333247304375
:02C9A400310060
:10C9A6004465766963652049443A2053544D3332D1
:10C9B60047303731206F722053544D333247303869
:02C9C60031003E
:10C9C8004465766963652049443A2053544D3332AF
:10C9D80047303531206F722053544D33324730364B
:02C9E80031001C
:10C9EA004465766963652049443A2053544D33328D
:10C9FA0047303331206F722053544D33324730342D
:02CA0A003100F9
:10CA0C004672656520737061636520666F72206382
:10CA1C006F66696775726174696F6E20696E2066E6
:10CA2C00616B6520454550524F4D3A20257520626B
:06CA3C00797465730A0025
:10CA42004D41585F504F535349424C455F4449460C
:10CA5200465F544F5F4D4541535552453A20257527
:02CA62000A00C8
:10CA640043616E6E6F742073746172742041444329
:0ECA740020696E20444D41206D6F64652100E5
:10CA820043616E6E6F7420636F70792056656374B4
:10CA92006F72205461626C652066726F6D20464C25
:10CAA20041534820746F2052414D2120444D412072
:0ECAB2006973206E6F742072656164792100D3
:10CAC00043616E6E6F742066696E69736820636F70
:10CAD0007079696E6720566563746F722054616265
:10CAE0006C652066726F6D20464C41534820746F10
:06CAF0002052414D21001F
:10CAF6004D6F646520302069732073656C656374BF
:10CB060065642E204175746F2D7265636F6E6E6558
:0ACB16006374206973204F4E2E0057
:10CB20004D6F646520312069732073656C65637493
:10CB300065642E204175746F2D7265636F6E6E652E
:0ACB40006374206973204F4E2E002D
:10CB4A004D6F646520322069732073656C65637468
:10CB5A0065642E204175746F2D7265636F6E6E6504
:0ACB6A006374206973204F4E2E0003
:10CB74004D6F646520332069732073656C6563743D
:10CB840065642E204175746F2D7265636F6E6E65DA
:0ACB94006374206973204F4E2E00D9
:10CB9E004D6F646520342069732073656C65637412
:10CBAE0065642E204175746F2D7265636F6E6E65B0
:0ACBBE006374206973204F4E2E00AF
:10CBC8004D6F646520352069732073656C656374E7
:10CBD80065642E204175746F2D7265636F6E6E6586
:0ACBE8006374206973204F4E2E0085
:10CBF200555020627574746F6E206973207072656F
:06CC0200737365642E004F
:02CC08004E00DC
:06CC0A00523A20257300E0
:10CC100043616E6E6F742073617665206461746128
:10CC200020696E20464C415348206D656D6F7279C6
:02CC30002100E1
:0ECC32004E4D49204552524F522121210A00F9
:02CC40000A00E8
:05CC42004D41494E00C8
:10CC470043616E6E6F742073746172742054494D22
:05CC57004552322100EE
:05CC5C001B5B324A00E1
:10CC610050726F6772616D20737461727465642EA6
:01CC710000C2
:10CC720043505520467265713A20257520487A0A3C
:01CC820000B1
:10CC830043616E6E6F74207265616420636F6E66BC
:10CC9300696775726174696F6E2066726F6D204685
:0DCCA3004C415348206D656D6F7279210082
:10CCB000257325733A204144432043616C696272B5
:10CCC0006174696F6E2076616C75653A2025750A0E
:01CCD0000063
:10CCD10043616E6E6F742073746F70204144432101
:01CCE1000052
:10CCE20025733A204441432043616C696272617446
:10CCF200696F6E2076616C756520666F722063685D
:0DCD0200616E6E656C20313A2025750A00C7
:10CD0F0025733A204441432043616C696272617418
:10CD1F00696F6E2076616C756520666F722063682F
:0DCD2F00616E6E656C20323A2025750A0099
:10CD3C0049742069732074696D6520746F20736168
:10CD4C00766520737461746973746963616C2064B3
:10CD5C0061746120696E20466C617368206D656D2D
:05CD6C006F72792E003A
:10CD7100496C6C6567616C204D6F64652069732037
:10CD810073656C65637465642E2044656661756CBA
:10CD910074204D6F646520342069732073656C6560
:10CDA100637465642E204175746F2D7265636F6EB7
:0DCDB1006E656374206973204F46462E00A6
:05CDBE00257325730040
:09CDC300493A20253564204100A5
:09CDCC004F56503A202531730046
:09CDD5004C56503A202531730040
:0DCDDE00543A202532642E256420B0430015
:10CDEB00095B2534645D2053616D706C656420763E
:10CDFB00616C7565733A20492B203D2025367520D3
:0DCE0B00202020492D203D202536750A00ED
:10CE180009094F66667365742076616C7565733AA7
:10CE280020492B203D20257520202020492D203DFC
:05CE38002025750A0031
:10CE3D0009094F66667365742076616C75653A20D5
:05CE4D002534640A0019
:10CE5200556E6B6E6F776E20636F6D6D616E6421C0
:01CE620000CF
:0DCE63005553415254206572726F722100C8
:04CE7000D1300008B5
:10CE740025733A205265766973696F6E206E756DFD
:0CCE84006265723A2030782534580A00AC
:10CE90004672656520737061636520666F722073EA
:10CEA00074617469737469637320696E2066616B61
:10CEB0006520454550524F4D3A20257520627974C2
:04CEC00065730A008C
:10CEC400435055207370656564206973206E6F74D8
:08CED4002036344D487A21009C
:10CEDC00466972737420737461727421205772697D
:10CEEC0074696E672064656661756C7420636F6E1F
:0CCEFC0066696775726174696F6E2100D1
:08CF08001B5B313B33326D006D
:10CF1000566563746F72205461626C65206861733A
:10CF2000206265656E20636F706965642066726F4C
:10CF30006D20464C41534820746F2052414D2E00C5
:10CF4000496C6C6567616C204D6F64652069732066
:10CF500073656C65637465642E2044656661756CE9
:10CF600074204D6F646520342069732073656C658F
:10CF7000637465642E204175746F2D7265636F6EE6
:0CCF80006E656374206973204F4E2E0014
:10CF8C00444F574E20627574746F6E206973207015
:08CF9C007265737365642E00D9
:08CFA4001B5B323B33306D00D2
:08CFAC002573207C2025730091
:0CCFB4005661623A20253464206D56005E
:0CCFC0005662623A20253564206D560050
:10CFCC001B5B323B33316D591B5B313B33326D0094
:08CFDC001B5B313B33366D0095
:08CFE400434847202D203100D5
:08CFEC00434847202D203000CE
:10CFF4000909566F6C746167652D64726F70204106
:10D0040044432076616C75653A202535642E0A0008
:10D0140009090946696E616C20766F6C74616765F5
:10D024002D64726F70204144432076616C75653ABB
:10D03400202534752E2046696E616C20766F6C74E1
:10D044006167652D64726F702076616C75653A2036
:08D05400253375206D560A001A
:10D05C0043616E6E6F742073617665206E65772008
:10D06C00534E20696E20464C415348206D656D6FC0
:04D07C0072792100A4
:10D0800043616E6E6F742073746172742054494DE5
:10D09000313720696E20495352206D6F646521003D
:08D0A0001B5B313B33316D00D5
:10D0A800486172646661756C74204552524F522112
:04D0B80021210A0028
:08D0BC001B5B323B33326D00B7
:08D0C4001B5B323B33336D00AE
:08D0CC001B5B323B33316D00A8
:04D0D4004D4F440078
:08D0D800010101030701000042
:08D0E00008040204080101012B
:10D0E8003031323334353637383941424344454696
:10D0F800FDF70008C006002038000000FDF7000812
:10D108000007002072080000FDF70008740F0020D7
:10D11800940500000FF800080000002040D1000826
:10D12800B90600000FF8000800600020F9D70008D1
:08D13800002000002BC40008D8
:10D140007047C04609480069C16A0E2905D8026BBC
:10D1500081600E2A06D8426170470F39026B8160E8
:10D160000E2AF8D90F3A42617047C046C007002026
:10D1700009480069C16A0E2905D8026B81600E2A30
:10D1800006D8426170470F39026B81600E2AF8D9C8
:10D190000F3A42617047C046C0070020F0B51A48F8
:10D1A0000069016B3A22194B9C5E194D2A6E1219C7
:10D1B000184EB242184F06DAB9421FD300230F228D
:10D1C000002B11D111E0012300220E291F4600D8A7
:10D1D00017462D6E2C19B44200DC13463B400E223C
:10D1E000D2430D4F002B00D089184161C16AB9426A
:10D1F00001D38160F0BD0F318160F0BD01230F22AA
:10D20000002BF1D1F1E7C046C0070020600E0020DE
:10D21000AC100020AC060000F10F0000F0B518487B
:10D220000069C16A3A22174B9C5E174D2A6E12198B
:10D23000164EB242164F03DA0E2912D8002311E01F
:10D2400001230022B9421F4600D317462D6E2C1928
:10D25000B44200DC13463B400F220D4F002B05D19A
:10D2600005E001230E22D243002B00D089188160F3
:10D27000016BB94201D34161F0BD0F314161F0BD95
:10D28000C0070020600E0020AC10002052090000F2
:10D29000F10F000009480069C26A09498A4205D3B2
:10D2A000036B82608B4206D3436170470F32036B7E
:10D2B00082608B42F8D20F3343617047C007002071
:10D2C000F10F000009480069C16A0E2905D8026BF8
:10D2D00081600E2A06D8426170470F39026B816067
:10D2E0000E2AF8D90F3A42617047C046C0070020A5
:10D2F00009480069C26A09498A4205D3036B826002
:10D300008B4206D3436170470F32036B82608B42BE
:10D31000F8D20F3343617047C0070020F10F0000BF
:10D3200009480069C16A0E2905D8026B81600E2A7E
:10D3300006D8426170470F39026B81600E2AF8D916
:10D340000F3A42617047C046C00700200948006993
:10D35000C26A09498A4205D3036B82608B4206D3B5
:10D36000436170470F32036B82608B42F8D20F33F8
:10D3700043617047C0070020F10F000009480069B1
:10D38000C26A09498A4205D3036B82608B4206D385
:10D39000436170470F32036B82608B42F8D20F33C8
:10D3A00043617047C0070020F10F00000248016A86
:10D3B000491C01627047C046A4110020B0B5154D4C
:10D3C0002889154CA080A0688047A8886989E060FA
:10D3D00021610D48016802220A430260E068216968
:10D3E000884200DC08464021084A515E884208D342
:10D3F0002168081820600649096C884203D96069D1
:10D40000804700202060B0BD04000240600E002074
:10D41000E4050020E81100200811002010B5124892
:10D420000069002181604161EA2210488152012196
:10D430000A030F4B1A60BFF34F8FBFF36F8F0D4A74
:10D440000D4B5366536F002B00D010BD0D4B197060
:10D4500041239B00C45A641CC45291670748006A68
:10D460000749486410BDC046C0070020600E002078
:10D4700080E100E0AC10002001000020A411002099
:10D48000E405002060110020F0B58BB0A1480068D1
:10D49000C469016801220A921207079209908768FD
:10D4A00023070891049756D0501C384001252A02C2
:10D4B000164620360E4006434DD00A40564256418D
:10D4C000E2070A9A00D03246002A07D109990D6274
:10D4D0008C2290498E582E438E5008993D406A42C6
:10D4E0006A41A6070A9E00D51646002E0AD10222DE
:10D4F00009990A628C2287498E58042737438F5036
:10D50000049F08996A426A4165070A9D04D4002D68
:10D5100004D0002B0ED41EE01500FAD10422099984
:10D520000A628C227B498D5802262E438E50089920
:10D53000002B10D5421E90418A060A9A00D402465A
:10D54000012A08D10820099908628C2271498B5858
:10D5500003438B5008990123D8050590200514D565
:10D560003846059A10409A060A4010180DD0D80285
:10D57000099908628820202266490A5084200A50AE
:10D58000089965480375654A83542020254606900E
:10D5900005402CD03846079A10400A46069E324075
:10D5A000024324D002934520C0005B4A13588826CA
:10D5B000584FBE59222E12D102990E02B3420ED2FA
:10D5C000D31809994E6A2727DE55544B0299D15436
:10D5D00013585B1C13500B460899049F07E00999E8
:10D5E0008869082202438A610899049F029B80206F
:10D5F00026460390064032D03846059A10400A4627
:10D60000039F3A4002432AD043480068842282584C
:10D61000212A14D1024656321788002F12D00768EB
:10D620000197076D02973F780092019A9762029ADC
:10D63000571C0765009A1088401E10800BE0006898
:10D64000026802E000680268039FBA430260026851
:10D65000402717430760304A232000011354402716
:10D660000A463A4050425041620600D50A900A9854
:10D6700000280ED109990868B8430860842025491C
:10D68000069A0A50264800220270882022240C5054
:10D690004A678C221F48805800282ED088242220D8
:10D6A0001C490A9408510899002D09D0049D029341
:10D6B000079B2B400D46069C25401D43029B1ED117
:10D6C000002E1AD0049A059D2A40039C2140114344
:10D6D00013D009990A68BA430A6084210D4A1D468D
:10D6E0001346069A5A500A99585026200A49002291
:10D6F0000A54232000010D545A670BB0F0BD09995C
:10D700008869082303438B610020024988500BB0CD
:10D71000F0BDC0461C100020240C00203102000087
:10D720004A0C002001000000FFFFFFFFC0E0FFFFE8
:10D7300001000000FFFFFFFF0100000002000000E9
:10D7400001000000FFFFFFFF0100000002000000D9
:10D7500001000000FFFFFFFF0100000004000000C7
:10D7600000DC0500FFFFFFFFC0E0FFFF0024F40026
:10D77000000000000202000000000002020202029B
:10D780000100000000000000000000000001010195
:10D790000001010001000202010100000000000080
:10D7A0000000000000000000000000000000000079
:10D7B0000000000000000000000000000000000069
:10D7C0000000000000000000000000000000000059
:10D7D0000000000000000000000000000001010146
:10D7E0000100010100000001010101000000000032
:10D7F000000000000000000000CDCDCDCDCDCDCD8E
:10D80000CDCDCDCDCDCDCDCDCDCDCDCDCDCDCDCD48
:10D81000CDCDCDCDCDCDCDCDCDCDCDCDCDCDCDCD38
:10D82000CDCDCDCDCDCDCDCDCDCDCDCDCDCDCDCD28
:10D83000CDCDCDCDCDCDCDCDCDCDCDCDCDCDCDCD18
:0CF7F000CDCDCDCDCDCDCDCDCD000000D8
:10F7FC00206861680834002200E042540139FCD5CD
:02F80C00704743
:10F80E0020686168A2680C3401E08B5C8354013A75
:04F81E00FBD570475F
:10F82200FFFFFFFFFFFFFFFFFFFFFFFFFFFFFFFFE6
:10F83200FFFFFFFFFFFFFFFFFFFFFFFFFFFFFFFFD6
:10F84200FFFFFFFFFFFFFFFFFFFFFFFFFFFFFFFFC6
:10F85200FFFFFFFFFFFFFFFFFFFFFFFFFFFFFFFFB6
:020000040801F1
:04EFFC008D650A43D2
:040000050800C475B6
:00000001FF
